:020000040000FA
:10000000F2EF03F01200FFFF04EF04F01200FFFF15
:10001000FFFFFFFFFFFFFFFF0CEF04F012000000E7
:100020000001776B1E0E716E0401400E096F200EE9
:100030000A6F040E0B6F880E086F0401200E0E6FFE
:10004000040E0F6F400E0C6F1200550EA76EAA0E15
:10005000A76EA68212000401226B010E236F12000C
:100060000001756B040121510001755D20E275C02E
:1000700000F0016A026A040122510024F36E235148
:100080000120F46E24510220F86EF4CFF7FFF3CF75
:10009000F6FF0800F5CF76F000017551EA6A250FEA
:1000A000E96E040EEA2276C0EFFF752BDBD7F86A03
:1000B0001200F00E04012217840EA66E0001756B6B
:1000C000040121510001755D26E27551EA6A250F90
:1000D000E96E040EEA22EFCF03F075C000F0016A6A
:1000E000026A040122510024F36E23510120F46EB0
:1000F00024510220F86EF4CFF7FFF3CFF6FF03C0D0
:10010000F5FF0C000F0E000175150F0801E19DDFD2
:100110000001752BD5D71200940EA66E0001756BE9
:10012000040121510001755D1EE27551006E016AE6
:10013000060ED89000360136E804FBE1026A01BEE3
:100140000268040122510024F36E23510120F46E51
:1001500024510220F86EF4CFF7FFF3CFF6FF75DFDE
:100160000001752BDDD7F86A1200A66A0001756BD5
:10017000040121510001755D10E2040122510001CA
:100180007525A96EA6807551EA6A250FE96E040EE1
:10019000EA22A8CFEFFF752BEBD712000001756B99
:1001A000040121510001755D15E204012251000195
:1001B0007525A96E7551EA6A250FE96E040EEA22CB
:1001C000EF50A86E040EA66E40DFA6B2FED7000167
:1001D000752BE6D71200C40EA66E0001756B0401E4
:1001E00021510001755D21E27551EA6A250FE96E22
:1001F000040EEA22EFCF03F075C000F0016A026A34
:10020000040122510024F36E23510120F46E245185
:100210000220F86EF4CFF7FFF3CFF6FF03C0F5FF2F
:100220000C0013DF0001752BDAD7F86A12008BD8A7
:10023000060E00017C5D03E36D50020B01E082D0ED
:100240000001770511E104010CBF0DD00401400E3F
:10025000096F400E040108170401087D880E04018F
:1002600008130001776B6ED0040108BF6BD000014A
:10027000756B04012051320A45E0CD0A34E0F80ADA
:100280002DE0020A26E0010A1FE0070A18E0010A31
:1002900011E0030A0AE0070A08E0060A01E041D07B
:1002A000DADE0001040E756F3DD0DADE050E0001C6
:1002B000752738D0FEDE0001010E756F33D02CDFBC
:1002C0000001010E756F2ED050DF050E000175275D
:1002D00029D064DF0001010E756F24D07CDF00019E
:1002E000010E756F1FD06D960001786B796B000160
:1002F0007807000E795B00017851791101E0F7D79A
:10030000FF0010D0030E0401215D03E10001010E86
:10031000756F040E0401215D03E10001010E756F8C
:1003200001D000D00001010E776F000175510AE085
:1003300075C00DF4400E04010C1704010C7D880EED
:1003400004010C131200060E00017C5D10E1000197
:100350007A517B1105E18B82200E7A6F4E0E7B6FF6
:10036000880E7A1904E1130E7B1901E18B920001CA
:100370007A07000E7B5B12006C5002E0000E01D089
:10038000010E00090BE0040100513C0BE842E84279
:100390000D0802E1D7EF01F0E0EF01F06C5002E050
:1003A000000E01D0010E040901E019D8120000016D
:1003B000606B616B666B676BB5EC02F062EF02F02D
:1003C000020E0001605D09E15CD8040100BD02D0AD
:1003D000C80E01D0880E006F1200A7EF02F0040EC5
:1003E00000017C5D09E112C46EFF6E50000802E25C
:1003F000050E01D0030E7C6F0001600509E10AD8EB
:10040000040104BD02D0C80E01D0880E046F120092
:10041000A7EF02F00001080E665D000E675903E2C7
:1004200066C069F002D0080E696F69C005F46951B1
:10043000006E016A0050665F0150675B180E646FC2
:10044000040E656F69511CE000017DA307D062C0F6
:10045000F6FF63C0F7FF0800F55005D062C0E9FF62
:1004600063C0EAFFEF5064C0E9FF65C0EAFFEF6ECA
:100470000001622B000E6323642B65236907E2D71A
:10048000120001C46AF000016A516625666F000E11
:100490006721676F180E626F040E636F6A5111E077
:1004A00062C0E9FF63C0EAFFEF5064C0E9FF65C0C6
:1004B000EAFFEF6E642B000E6523622B63236A074D
:1004C000EDD71200000161510BE10401080E016F2C
:1004D000100E026F040E036F840E006F040123D010
:1004E000040110AF22D0000166510401165D000125
:1004F00067510401175904E216C466F017C467F087
:1005000089DF0001010E606F0401080E016F100EFB
:10051000026F040E036F800E006F0401180E066F49
:10052000040E076FC80E046F10D00001020E606F3A
:100530000401056BC80E046F0401080E016F180E4C
:10054000026F040E036FC80E006F6D981200000159
:10055000606B0401080E016F100E026F040E036F32
:10056000880E006F0401046B120004011051600B2F
:10057000E842E842E842E842E842000901E01200AD
:100580001151080A39E0010A35E00F0A0AE0030AAE
:1005900001E012000001010E616F0001040E7C6F8A
:1005A00012000001010E616F0401130507E1000153
:1005B0007E0E626F070E636F120E13D0020E135D74
:1005C00007E10001900E626F070E636F200E09D0E5
:1005D000030E135D0AE10001B00E626F070E636F38
:1005E000040E0001666F676B02D00001616B0001B1
:1005F0007D8312000AEF03F00001010E616F00011C
:100600007E0E626F000E636F00017D930001010E8C
:10061000666F12000001010E616F12C47EF00401CA
:10062000125104E10001050E7C6F12000001060E5C
:100630007C6F10EF00F0080E6D6E6DBAFED7686A21
:10064000110E696E0001020E7C6F12006850040BDF
:1006500006E06950040B03E06D9269946894685059
:10066000010B04E06950010B01E027D86850100B22
:1006700009E06950100B06E0698468986D82A08AD1
:100680000300A19A6850200B09E06950200B06E096
:1006900070A003D0A7EC02F07090689A030E0001DE
:1006A0007C5D01E209D06850080B06E06950080B38
:1006B00003E0BCEC01F068961200686A7B0E696E7C
:1006C0006E6A160E706E68A602D06896FCD76D989A
:1006D000A7EC02F000017E6B0001030E7C6F12009C
:1006E0001E0EF66E000EF76E000EF86E0001090089
:1006F000F550706F0900F550716F03E1706701D01C
:100700003DD00900F5506B6F0900F5506C6F090082
:10071000F5506D6F09000900F550E96E0900F550BC
:10072000EA6E090009000900F5506E6F0900F550E6
:100730006F6F09000900F6CF72F0F7CF73F0F8CFB2
:1007400074F06BC0F6FF6CC0F7FF6DC0F8FF0001DE
:100750006E5302E16F5307E00900F550EE6E6E072D
:10076000F8E26F07F9D772C0F6FF73C0F7FF74C0E5
:10077000F8FF00017007000E715BBFD71200120175
:10078000000200000008D8040B0000000000000177
:10079000090220000101008032090400000200006B
:1007A000000007050102400000070581024000002B
:1007B00004030904C1CF80F00F0EC11282A404D03B
:1007C00080C0C1FF00EF04F0FC0E8B16FC0E9416E7
:1007D000140E6F6E1BEC03F026EC03F017EC01F027
:1007E000FBD7120013EE00F023EE00F0F86A059C30
:1007F00070EC03F0DAEC03F0FDD71200FFFFFFFF0F
:1008000025EF30F01200FFFFFDEF04F01200FFFFB4
:10081000FFFFFFFFFFFFFFFF1CEF04F01200FFFFD1
:10082000FFFFFFFFFFFFFFFFFFFF0100AB5C0000CA
:100830007D00000001000000D8CFE4FFE0CFE4FF1E
:10084000E46EDACFE4FFE2CFDAFFE9CFE4FFEACFEC
:10085000E4FFF6CFE4FFF7CFE4FFF5CFE4FFF3CFFB
:10086000E4FFF4CFE4FFFACFE4FF00EE17F0100E40
:10087000E80403E3EECFE4FFFBD700EE27F0100E11
:10088000E80403E3EECFE4FFFBD7E652F2A42ED058
:10089000F294280EE66EF10EE66EA3EC2FF0E55210
:1008A000E552005012E00CC037F00DC038F00C06D5
:1008B000000E0D5A3750381008E1010E156E10C0A9
:1008C0000CF011C00DF04FEC30F002019A510EE027
:1008D0000EC037F00FC038F00E06000E0F5A37501A
:1008E000381004E1320E0E6E0F6A8B729EAC36D059
:1008F0009E9C8B7284EC2FF0F3CF12F0F4CF13F0A8
:100900000050FF0A0CE0FE0A05E0010A01E008D0F1
:10091000156A07D0156A0C6A0D6A006A02D001D008
:10092000000601A002D002018D2B01A217D000C049
:1009300020F202C021F212C022F2000E1214376E11
:10094000FF0E1314386E38C037F0386A37C023F200
:1009500002017E0E246F67EC0CF0022AF2A024D074
:10096000F2900750086E8150076E08500718096E04
:1009700002018F51091418E08F5107140BE0920502
:1009800006E1550EE66E94EC0FF0E55202D0B8EC9D
:100990000FF00AD0920503E1B8EC0FF005D0550E28
:1009A000E66E94EC0FF0E552E55200EE36F0100ED4
:1009B000E80403E3E5CFEDFFFBD700EE26F0100ED1
:1009C000E80403E3E5CFEDFFFBD7E5CFFAFFE5CF82
:1009D000F4FFE5CFF3FFE5CFF5FFE5CFF7FFE5CF78
:1009E000F6FFE5CFEAFFE5CFE9FFE5CFDAFFE55017
:1009F000E5CFE0FFE5CFD8FF1000DACFE4FFE2CF8C
:100A0000DAFFE652E552E5CFDAFF1100D9CFE6FF73
:100A1000E1CFD9FF020EE126146A156A006A016A65
:100A200002018D6B046A320E0E6E0F6A010E9A6F10
:100A30009B6B166A9D6B00017D6B0201466B476BD9
:100A4000486B496B100E8F6F080E906F926B010E02
:100A5000936F070EB46EB56AC26A0F0EC16E896AD3
:100A6000010E926E8A6A936A050E816E3C0E8B1699
:100A70009416FC0E8B16941610C00CF011C00DF0DD
:100A8000DE6ADD6ADECF27F0DDCF28F0060E275CB8
:100A9000000E28580EE2DECFE9FFDDCFEAFFE40EBC
:100AA000E926020EEA22EF6ADF2A010E01E3DB2AC1
:100AB000E9D706EC26F0800EE66E03EC27F0E5524F
:100AC000E66A03EC27F0E552890EE66E020EE66E4A
:100AD000050EE66EDBEC0DF0E552E552E552FF083F
:100AE00003E10201080E896F0201150E8A6F3FECC7
:100AF0000DF08BC2E4F22DEC0FF0990EE66E020EB3
:100B0000E66E240EE66EDBEC0DF0E552E552E552A2
:100B1000FF0803E10201030E996F940EE66E020EC8
:100B2000E66E470EE66EDBEC0DF0E552E552E5525F
:100B3000FF0803E10201010E946F950EE66E020EAE
:100B4000E66E250EE66EDBEC0DF0E552E552E55261
:100B5000FF0803E10201050E956F880EE66E020E96
:100B6000E66E060EE66EDBEC0DF0E552E552E55260
:100B7000FF0803E10201090E886F02010C0E8A6F63
:100B80003FEC0DF0FF0E02018B5D0AE01F0E8B158E
:100B9000856FE00E8B15E00BE838E840866F03D0D8
:100BA000010E856F866F4A0EE66E020EE66E070E28
:100BB000E66E5DEC0DF0E552E552E552FF0809E105
:100BC0000201400E4A6F590E4B6F730E4C6F070EA9
:100BD0004D6F520EE66E020EE66E100EE66E5DEC86
:100BE0000DF0E552E552E552FF0806E10201220E42
:100BF000526F536B546B556B960EE66E020EE66E9B
:100C0000160EE66EDBEC0DF0E552E552E552FF08FC
:100C100002E10201966B620EE66E020EE66E2E0E89
:100C2000E66E5DEC0DF0E552E552E552FF0805E198
:100C30000201626B636B646B656B660EE66E020E9F
:100C4000E66E320EE66E5DEC0DF0E552E552E552D1
:100C5000FF0805E10201666B676B686B696B6A0EE2
:100C6000E66E020EE66E4A0EE66E5DEC0DF0E552A3
:100C7000E552E552FF0808E10201980E6A6FA60EE0
:100C80006B6F6B0E6C6F6D6B6E0EE66E020EE66E2A
:100C90004E0EE66E5DEC0DF0E552E552E552FF08B2
:100CA00008E10201980E6E6FA60E6F6F6B0E706FEB
:100CB000716B720EE66E020EE66E520EE66E5DEC23
:100CC0000DF0E552E552E552FF0808E10201800E01
:100CD000726F960E736F980E746F756B760EE66E6C
:100CE000020EE66E200EE66E5DEC0DF0E552E5526A
:100CF000E552FF0808E10201980E766FA60E776FA5
:100D00006B0E786F796B970EE66E020EE66E600ED4
:100D1000E66EDBEC0DF0E552E552E552FF0803E12B
:100D20000201440E976F420EE66E020EE66E1C0E36
:100D3000E66E5DEC0DF0E552E552E552FF0805E187
:100D400002014269436944694569BDD977EC16F0EF
:100D50008E0EE66E020EE66E370EE66EDBEC0DF0E2
:100D6000E552E552E552FF0803E10201800E8E6F65
:100D7000050EE66E000EE66E360EE66EDBEC0DF04E
:100D8000E552E552E552FF0801E1056AB8EC0FF0C3
:100D9000870EE66E020EE66E3C0EE66EDBEC0DF0A4
:100DA000E552E552E552FF0802E10201876B87C276
:100DB000E4F27AEC0CF0140EE66EBFEC2FF0E55284
:100DC000280EE66EF10EE66EA3EC2FF0E552E5522A
:100DD000D08ED59EF28AF194F190F28EF28CD58E5F
:100DE000010E146E8A9A8B92020EE15C02E2E16AB5
:100DF000E552E16EE552E7CFD9FF1200D9CFE6FF09
:100E0000E1CFD9FF030EE126DF6A060E0201FC5D89
:100E100003E36D50020B01E020D1050EE66E000EDB
:100E2000E66E020EE66E03EC29F0E552E552E5525D
:100E3000DF6EDFCF27F0000EE76E2718E8AE02D096
:100E4000273403D0E750D880275401E302D1010EA4
:100E5000DB6A020EDB6A010EDBCF27F0020EDBCF6E
:100E600028F0D890285004E6050E275C000E28587C
:100E70001FE2010EDBCFE9FF020EDBCFEAFF000E1F
:100E8000E926020EEA22EF50E66E010EDBCFE9FF03
:100E9000020EDBCFEAFFE40EE926020EEA22E5525B
:100EA000E750EF6E010EDB2A020E01E3DB2AD3D7F7
:100EB0000201E851FF0A01E1C8D0010A01E1C2D0F4
:100EC000030A01E1BCD0010A01E1B6D0070A01E141
:100ED000B0D0010A01E1AAD0030A01E1A4D0710A4D
:100EE00001E19DD00F0A01E196D0010A01E18FD006
:100EF000030A01E187D0010A01E180D0070A01E17C
:100F000079D0010A73E0030A6DE0010A67E0FF0A85
:100F100062E0010A5DE0030A58E0010A53E0070AB3
:100F20004EE0010A49E0030A44E0010A3FE00F0AEB
:100F30003AE0010A35E0020A30E07D0A2CE0010ABD
:100F400028E00F0A24E0010A1FE0030A1BE0010A5F
:100F500017E0070A13E0010A0CE0030A06E0010AA1
:100F600001E076D007EC0DF074D0046BE86BE0D8AC
:100F700070D0010E046FE86FDBD86BD0F5D969D063
:100F800059DA67D0ADDA65D03AEC0CF062D0EEDB1E
:100F900060D0ECDB5ED06CDB5CD08FEC27F059D0FE
:100FA0000EEC22F056D0A3EC1FF053D06AEC1CF0EC
:100FB00050D0F3EC0FF04DD0ACEC1AF04AD0D2EC9C
:100FC0000FF047D077EC0FF044D020EC0DF041D07B
:100FD000B8EC0EF03ED07AEC0CF03BD0010E886FEE
:100FE0003ED937D0020E886F3AD933D0030E886FBE
:100FF0005AD92FD0040E886FD4D92BD0050E886F04
:101000002DDA27D0060E886F09EC0CF022D0070EDF
:10101000886F90DB1ED0080E886F8CDB1AD0090E0B
:10102000886F73DA16D0FDEC24F013D02DEC16F097
:1010300010D056EC16F00DD0D6EC0EF00AD02DECF8
:101040000FF007D06DEC0EF004D0EBEC0CF001D0FB
:101050006FD802018D5101E08D6B030EE15C02E25D
:10106000E16AE552E16EE552E7CFD9FF12000201D5
:101070008851060A24E00E0A20E00F0A1CE00E0A3E
:1010800018E00C0A14E0010A10E0070A0CE0010A5B
:1010900006E0030A01E015D0E86B4AD813D0010E30
:1010A000E86F46D80FD060D90DD0C4D90BD018DA6C
:1010B00009D0DEDA07D05ADB05D058DB03D0DADB03
:1010C00001D036D8120002018851060A2CE00E0A1F
:1010D00028E00F0A24E00E0A1EE00C0A1AE0010ABA
:1010E0000DE0070A09E0010A05E0030A01E01DD04E
:1010F000B6D81DD0B4D81BD0D6D819D08551080D7C
:10110000F3CFE4F2F80EE415E46F060EE41349D9C8
:101110000ED0A4D90CD0010EE46FF7D908D00ADBA9
:1011200006D008DB04D075DB02D0010E9C6F1200E4
:101130008B728A9AE7C241F214D8E6C241F211D802
:10114000E5C241F20ED8E4C241F20BD8E8C241F246
:1011500008D88A8AC80EE66E33EC30F0E5528A9AD7
:101160001200D9CFE6FFE1CFD9FF020EE1268A9C1B
:10117000DE6ADD6ADECF27F0DDCF28F0D890285078
:1011800004E6080E275C000E285817E241C227F03B
:10119000286A27BE2868010E2714E8B08A8EE8A0C6
:1011A0008A9E8A8CCCD88A9C020141914143C7D83F
:1011B000DF2A010E01E3DB2ADDD7020EE15C02E249
:1011C000E16AE552E16EE552E7CFD9FF1200D9CFCF
:1011D000E6FFE1CFD9FF050EE126800EF36E040E87
:1011E000F3CFDBFF8A9C010EF36E020EF3CFDBFF21
:1011F000030EDB6ADE6ADD6ADECF27F0DDCF28F082
:10120000D890285004E6080E275C000E28581DE2EE
:101210008A9E040EDB500201411501E08A8E010E08
:10122000F36E020EF3CFDBFF030EDB6A8A8C87D8E6
:101230008A9C040EDBCFF3FFF390F342F3CFDBFF86
:10124000DF2A010E01E3DB2AD7D7050EE15C02E2BB
:10125000E16AE552E16EE552E7CFD9FF12000201E3
:10126000010E9C6F8B728A8C6AD88A9C68D88A8A95
:1012700066D88A9A0201A80E416F73DF0201A50E9B
:10128000416F6FDF0201080E416F6BDF02010A0E32
:10129000416F67DF0201010E416F63DF50D88A8A18
:1012A0004ED88A9A12000201010E9C6F140EE66E4F
:1012B00033EC30F0E552898A140EE66E33EC30F0F0
:1012C000E552899A140EE66E33EC30F0E552898AC5
:1012D000140EE66E33EC30F0E552899A0201070EE7
:1012E000416F75DF0201100E416F71DF0201200EA8
:1012F000416F6DDF0201416B6ADF0201400E416FF9
:1013000066DF898A1E0EE66E33EC30F0E552899A6C
:101310000201070E416F5BDF0201100E416F57DFC4
:101320000201200E416F53DF0201416B50DF0201C9
:10133000400E416F4CDF8A8A02D88A9A1200D9CFB8
:10134000E6FFE1CFD9FF020EE126010EDE6EDD6A77
:10135000020EDE6EDD6AE15C02E2E16AE552E16EF8
:10136000E552E7CFD9FF1200898AE9DF899A0201A5
:10137000020E416F2CDFE4C241F229DFE5C241F2E7
:1013800026DFE6C241F223DFE7C241F220DF02019D
:10139000416B1DDF0201416B1ADF8A8AD0DF8A9A16
:1013A0001200D9CFE6FFE1CFD9FF020EE1260201FC
:1013B000010E9C6FDE6ADD6ADECF27F0DDCF28F0FC
:1013C000296AD8902950000A06E6600E275CEA0ECA
:1013D0002858000E295806E2416BDF2A010E01E36E
:1013E000DB2AEAD7898A899A010E416FF0DE020171
:1013F000416BEDDE0201416BEADEE4C241F2E7DE61
:101400008A8A9DDF8A9A0201416BE1DEE0DEDFDE3F
:10141000DEDE0201420E416FDADE8A8A90DF8A9AAE
:10142000020EE15C02E2E16AE552E16EE552E7CFCD
:10143000D9FF12000201040E416FC9DEE4C241F27D
:10144000C6DEE5C241F2C3DEE6C241F2C0DEE7C25B
:1014500041F2BDDE8A8A73DF8A9A12000201010E10
:101460009C6F416FB4DE0201900E416FB0DE02014D
:10147000416BADDE0201416BAADE320EE66E41EC3D
:1014800030F0E5520201416BA2DE0201800E416F95
:101490009EDE0201050E416F9ADE0201200E416FB1
:1014A00096DE0201416B93DE0201416B90DE020188
:1014B000F00E416F8CDE0201040E416F88DE0201E6
:1014C000200E416F84DE0201416B81DE0201416B1F
:1014D0007EDE0201416B7BDE8A8A31DF8A9A12004E
:1014E0000201010E9C6F040E416F71DEE4C241F2F5
:1014F0006EDEE5C241F26BDEE6C241F268DEE7C2B3
:1015000041F28A8A1CDF8A9A1200D9CFE6FFE1CF26
:10151000D9FF020EE1260201010E9C6F8A9ADE6A53
:10152000DD6ADECF27F0DDCF28F0296AD890295078
:10153000000A06E6600E275CEA0E2858000E2958BD
:1015400006E2416BDF2A010E01E3DB2AEAD7E4C29F
:1015500027F0286A27BE286827C0DEFF28C0DDFFE5
:10156000416B35DE0201120E416F31DE0201010EC8
:10157000416F2DDE8A8AE3DE8A9AE4C227F0286A68
:1015800027BE286827C0DEFF28C0DDFF0201416BAF
:101590001EDE0201200E416F1ADED9CFE9FFDACF3D
:1015A000EAFF030ED880EE54000EED5419E2D9CFB5
:1015B000E9FFDACFEAFF040EEE1801E1ED5003E196
:1015C0000201416B0CD0DECF27F0DDCF28F0D890A0
:1015D00028322732D8902832273227C041F202D051
:1015E0000201416BF4DD8A8AAADE8A9A0201416B0C
:1015F000EEDD0201220E416FEADDD9CFE9FFDACF3D
:10160000EAFF030ED880EE54000EED5404E202010E
:10161000850E416F03D00201020E416FD8DD8A8A28
:101620008EDE8A9A0201416BD2DD0201100E416FFB
:10163000CEDDD9CFE9FFDACFEAFF030ED880EE5432
:10164000000EED5404E20201800E416F03D002014E
:10165000900E416FBCDD8A8A72DE8A9A020EE15CCE
:1016600002E2E16AE552E16EE552E7CFD9FF1200EE
:101670000201410E416FABDD0201AB0E416FA7DDF0
:10168000E4C241F2A4DDE5C241F2A1DDE6C241F2CD
:101690009EDD8A8A54DE8A9A0201410E416F97DDEF
:1016A0000201A80E416F93DDE7C241F290DD020115
:1016B000416B8DDD8CDD8A8A42DE8A9A1200D9CF99
:1016C000E6FFE1CFD9FF050EE126800EF36E040E92
:1016D000F3CFDBFFDE6ADD6ADECF27F0DDCF28F057
:1016E000D890285004E6080E275C000E285817E210
:1016F000040EDB500201411502E08A8E01D08A9E61
:101700008A9C1DDE8A8C040EDBCFF3FFF390F3423C
:10171000F3CFDBFFDF2A010E01E3DB2ADDD78A9E50
:10172000050EE15C02E2E16AE552E16EE552E7CFC7
:10173000D9FF120002019C6B8A8C8A8A00DE8A9A89
:101740000201210E416FBBDF0201416BB8DF8A8AC3
:10175000F6DD8A9A0201200E416FB1DF0201416B72
:10176000AEDF8A8AECDD8A8A8A8C1200D9CFE6FF46
:10177000E1CFD9FFE6528A9A3F0E0201E615416F8A
:10178000400E4111416F9BDFE7C241F298DF8A8A28
:10179000D6DD8A9A060EE5C2E7FF070B04E0E742B2
:1017A000E79EE806FCE1E750DF6E030EDF1402015E
:1017B000416FE451040DF350DF6E3C0EDF14DF6E19
:1017C000DF504111416F400E4111416F78DF060E2D
:1017D000E6C2E7FF070B04E0E742E79EE806FCE10C
:1017E000E750DF6E030EDF140201416FE551040D77
:1017F000F350DF6EFC0EDF14DF6EDF504111416FDE
:101800005EDF8A8A9CDD8A8CE552E552E7CFD9FFFC
:1018100012000201010E9C6F8A8C8A8A90DD8A9ADE
:101820000201D80E416F4BDF0201416B48DF8A8A0B
:1018300086DD8A9A0201900E416F41DF0201416B01
:101840003EDF8A8A7CDD8A9A0201600E416F37DFB3
:101850000201416B34DF8A8A72DD8A9A0201C00E6E
:10186000416F2DDF0201416B2ADF8A8A68DD8A8A97
:101870008A8C1200D9CFE6FFE1CFD9FFE6528A9ACF
:101880000201300E416F1BDFE7C241F218DF020197
:10189000210E416F14DFE6C241F211DF8A8A4FDD6B
:1018A0008A9A0201320E416F0ADFE5C241F207DF78
:1018B0000201230E416F03DFE4C241F200DF8A8A96
:1018C0003EDD8A8CE552E552E7CFD9FF120004AE27
:1018D00010D0000161510DE10001200E626F020E77
:1018E000636F0001050E666F0001676B0001010E5A
:1018F000616F1200D9CFE6FFE1CFD9FF060EE126D6
:101900008A9E899889943F0E0201E415876F87515A
:10191000E66ED950040FE96EDACFEAFFE552E750E0
:10192000EE6EED6AE70543E0DE6ADD6ADECF27F0A2
:10193000DDCF28F0D890285004E6060E275C000E74
:10194000285830E2200EE76E040EDBCF27F0050E9C
:10195000DBCF28F0E7502716286A020E27C0DBFFEE
:10196000030E28C0DBFFD950020FE96EDACFEAFF81
:10197000EE50ED1002E08A8E01D08A9EE0DC89886C
:10198000DEDC8998D950040FE96EDACFEAFF010E48
:10199000D890EE36ED36E806FBE1DF2A010E01E3D2
:1019A000DB2AC4D7CCDC8984CADC89948A9E87C2AE
:1019B00020F20201216B226B03C223F27F0E246FFF
:1019C00086DF060EE15C02E2E16AE552E16EE55275
:1019D000E7CFD9FF1200D9CFE6FFE1CFD9FF020E42
:1019E000E1268B708B72E66A04C2E6FF010EE66E9A
:1019F00009EC21F0E552E552E552020EE15C02E20B
:101A0000E16AE552E16EE552E7CFD9FF120002012B
:101A10008A6B35D88BC220F202018A2B30D88BC258
:101A200021F202018A2B2BD88BC222F20201060E70
:101A30008A6F25D88BC223F20201246B67EF0CF06A
:101A400000C220F201C221F20201236B04C224F27F
:101A500001C28AF2020E005D0DE102C28CF216D8BC
:101A60000ED802018C518B5D02E0236B02D0010E77
:101A7000236F01D004D88BC222F267EF0CF0A69E30
:101A80008AC2A9FFA680A8CF8BF2120002019B5147
:101A900013E0A69EA6848AC2A9FF8CC2A8FF145098
:101AA00001E0F29E550EA76EAA0EA76EA682A1A80F
:101AB000FED7145001E0F28E1200D9CFE6FFE1CF3D
:101AC000D9FF060EE126020EDB6A030EDB6A040E66
:101AD000DB6A050EDB6AFE0EDB50030F02018A6F24
:101AE000010EDE6EDD6ADECF27F0DDCF28F0D89064
:101AF000285004E6050E275C000E285828E2D9502D
:101B0000020FE96EDACFEAFFEF50EE6AEFCFF4FF93
:101B1000EE6EEF50F4CFEEFFEF6EB1DF8BC227F029
:101B2000286A296A2A6AD950020FE96EDACFEAFFD9
:101B30002750EE122850EE122950EE122A50EE12C3
:101B400002018A07DF2A010E01E3DB2ACCD7D95034
:101B5000020FE96EDACFEAFFE868EE1808E1E868FC
:101B6000EE1805E1E868EE1802E1E868EE1803E116
:101B7000FF0E15D014D0FC0EDBCFE9FFFD0EDBCF3E
:101B8000EAFF020EDBCFEEFF030EDBCFEEFF040E0B
:101B9000DBCFEEFF050EDBCFEEFF000E00D0276E91
:101BA000060EE15C02E2E16AE552E16E2750E55281
:101BB000E7CFD9FF1200D9CFE6FFE1CFD9FFFE0E64
:101BC000DBCF8AF25CDFFF0E02018B5D03E1FF0ECB
:101BD0000BD00AD0FC0EDBCFE9FFFD0EDBCFEAFF16
:101BE0008BC2EFFF8B5100D0E552E7CFD9FF120037
:101BF000D9CFE6FFE1CFD9FF080EE126FE0EDBCFFD
:101C00008AF2FC0EDBCFE9FFFD0EDBCFEAFF040E0C
:101C1000EECFDBFF050EEECFDBFF060EEECFDBFFD8
:101C2000070EEECFDBFFDE6ADD6ADECF27F0DDCF09
:101C300028F0D890285004E6040E275C000E28589F
:101C400040E2040EDBCF27F0050EDBCF28F0060EB6
:101C5000DBCF29F0070EDBCF2AF0275002018C6F73
:101C600015DFD950040FE96EDACFEAFF080EE76EF0
:101C7000D890030EEB32020EEB32010EEB32EF3254
:101C8000E706F6E102018A2B020EDB6A030EDB6A2D
:101C9000020EDBCF27F0030EDBCF28F0D8902850C0
:101CA00004E6D00E275C070E285806E2020EDB2A57
:101CB000030E01E3DB2AECD7DF2A010E01E3DB2A66
:101CC000B4D7276E080EE15C02E2E16AE552E16EEC
:101CD0002750E552E7CFD9FF1200D9CFE6FFE1CF79
:101CE000D9FF020EE126DE6ADD6A00C203F002C2FD
:101CF00027F0286A27BE286827C0DEFF28C0DDFF3E
:101D0000DECF10F0DDCF11F010C011F0106A000E20
:101D10001016FF0E111602010151DE6EDD6ADE5053
:101D20001012DD50111203C201F00B0EE66E040E0C
:101D3000E66EF90EE66EDDEC2EF0E552E552E55268
:101D400003C020F210C021F211C027F0286A27C07A
:101D500022F201C023F204C224F2B9DD020EE15CDA
:101D600002E2E16AE552E16EE552E7CFD9FF1200E7
:101D700000C200F0FF0E0201015D02E001C202F0AC
:101D800002C203F003C201F0006B005106E04CEC0C
:101D900030F0156A0C6A0D6A08D0010E156E10C07D
:101DA0000CF011C00DF04FEC30F01200D9CFE6FF6F
:101DB000E1CFD9FF020EE126010EDB6AFF0E020120
:101DC000005D04E1DE52010EDD6E2CD0005103E116
:101DD000056A87D827D001C28EF200C205F0010E35
:101DE000051407E0100E041404E0100E8F6F6ED877
:101DF00002D08F6B76D802018EA503D0010E926FB0
:101E000001D0926B020E051406E0100E041403E0DC
:101E1000080E906F01D0906B8EAF03D0010E936FC0
:101E200001D0936B05C020F2010EDB0402E1020138
:101E3000208B8EC221F20AC022F204C023F20201DA
:101E4000FC0E246F44DD020EE15C02E2E16AE55221
:101E5000E16EE552E7CFD9FF1200D9CFE6FFE1CF1F
:101E6000D9FFE652E4C2DFFF280EDF1403E1DF50A2
:101E7000046E02D0400E046E04AC04D00201010EC8
:101E80009A6F03D002019A6B8B9205C000F28EC24A
:101E900001F28CDF04A004D00201010E9B6F02D07E
:101EA00002019B6BD70E0416150E8A6FEFDD04C07E
:101EB00020F28BC221F20201226B236BFD0E246FF4
:101EC00006DDE552E552E7CFD9FF120002018F513E
:101ED0009312FE0EE66EDBEC2FF0E552F286F190E7
:101EE0001200936AF296F290F296F18E1200800E32
:101EF000051480080EE1AA0E0201005D08E1550EEE
:101F0000015D05E1AA0EE66E0FD8E55201D030D88A
:101F10000AD0E6687C0EE66E030EE66E09EC21F050
:101F2000E552E552E5521200D9CFE6FFE1CFD9FFE5
:101F3000010E166E100E041409E0020E051406E0E0
:101F40000201930502E18A8601D08A96CAEC16F056
:101F5000FE0EDBCFE6FF7C0EE66E030EE66E09ECAE
:101F600021F0E552E552E552E552E7CFD9FF1200E4
:101F7000166A100E041409E0020E051406E00201B0
:101F8000930502E18A9601D08A86CAEC16F0E66AC9
:101F90007C0EE66E030EE66E09EC21F0E552E5528A
:101FA000E5521200D9CFE6FFE1CFD9FFE652DF6A52
:101FB0000201E50513E1F80E8116070EE415DF6E48
:101FC000DFCF95F2DF508112E66A04C2E6FF010E10
:101FD000E66E09EC21F0E552E552E552E552E55294
:101FE000E7CFD9FF1200D9CFE6FFE1CFD9FF080E26
:101FF000E126010EDE6EDD6A9EEC21F046C276F22D
:1020000047C277F248C278F249C279F276C25AF2F0
:1020100077C25BF278C25CF279C25DF2CAEC16F06C
:102020005EC246F25FC247F260C248F261C249F244
:10203000D9CFE9FFDACFEAFF010EEE1801E1ED504A
:1020400008E1800EF36E020EF3CFDBFF030EDB6AB6
:1020500004D0020EDB6A030EDB6A020EDBCFE6FF62
:10206000790EE66E020EE66E09EC21F0E552E552BD
:10207000E552080EE15C02E2E16AE552E16EE552EA
:10208000E7CFD9FF1200D9CFE6FFE1CFD9FF060E87
:10209000E126DE6ADE6A010EDE6EDD6ADD52DD52A9
:1020A0000201D66FD76BD86BD96BA60EE96E020E04
:1020B000EA6EBA51EE5CBB51EE58BC51EE58BD51C0
:1020C000EE5812E3CA69CB69CC69CD69CE69CF6994
:1020D000D069D169D651D711D811D91104E0D66988
:1020E000D769D869D96963D2BAC2E6FFBBC2E6FF35
:1020F000BCC2E6FFBDC2E6FF98DAE552E552E55202
:10210000E552040EF3CFDBFF050EF4CFDBFF040E28
:10211000DB501F0B08E00201D890BA37BB37BC3741
:10212000BD37E806F9E1100E1F0BBAC2BEF2BBC202
:10213000BFF2BCC2C0F2BDC2C1F208E00201D89039
:10214000C133C033BF33BE33E806F9E1BAC2C2F2CD
:10215000BBC2C3F2BCC2C4F2BDC2C5F20201C46BB1
:10216000C56B040EDB501F0BA6C227F0A7C228F0D8
:10217000A8C229F0A9C22AF007E0D890273628364D
:1021800029362A36E806F9E1040EDBCF2FF0050EDA
:10219000DBCF30F0200ED8802F56000E30562F5057
:1021A0001F0BAAC22BF0ABC22CF0ACC22DF0ADC2FB
:1021B0002EF007E0D8902E322D322C322B32E8064A
:1021C000F9E127502B100201AE6F28502C10AF6F91
:1021D00029502D10B06F2A502E10B16F040EDB5015
:1021E0001F0BAAC2B6F2ABC2B7F2ACC2B8F2ADC214
:1021F000B9F208E00201D890B637B737B837B93727
:10220000E806F9E1100E1F0BB6C29EF2B7C29FF2AC
:10221000B8C2A0F2B9C2A1F208E00201D890A1337D
:10222000A0339F339E33E806F9E1B6C2A2F2B7C2EB
:10223000A3F2B8C2A4F2B9C2A5F20201A46BA56BC5
:10224000AEC21DF0AFC21EF0B0C21FF0B1C220F08E
:10225000BEC222F0BFC223F0C0C224F0C1C225F02A
:1022600060EC2FF01DC0CAF21EC0CBF21FC0CCF232
:1022700020C0CDF2CAC21DF0CBC21EF0CCC21FF0EE
:10228000CDC220F0BEC222F0BFC223F0C0C224F0F3
:10229000C1C225F0A5EC2EF019500201AE5DDA6F37
:1022A0001A50AF59DB6F1B50B059DC6F1C50B1593D
:1022B000DD6FD9CFE9FFDACFEAFFEE50CA5DEE500D
:1022C000CB59EE50CC59EE50CD593DE2DAC21DF05B
:1022D000DBC21EF0DCC21FF0DDC220F0DFCF22F037
:1022E000010EDBCF23F0020EDBCF24F0030EDBCF99
:1022F00025F0A5EC2EF0195002019E25276E1A50EC
:102300009F21286E1B50A021296E1C50A1212A6EEE
:10231000CAC21DF0CBC21EF0CCC21FF0CDC220F04D
:10232000C2C222F0C3C223F0C4C224F0C5C225F049
:10233000A5EC2EF01950275C1A5028581B5029582C
:102340001C502A5824E20201CA07000ECB5BCC5B6A
:10235000CD5BBE0EE96E020EEA6EDA51EE24DA6F44
:10236000DB51EE20DB6FDC51EE20DC6FDD51EE2027
:10237000DD6FD9CFE9FFDACFEAFFEE50DA5DEE503C
:10238000DB59EE50DC59EE50DD5901E292D7AEC276
:102390001DF0AFC21EF0B0C21FF0B1C220F0DFCFFF
:1023A00022F0010EDBCF23F0020EDBCF24F0030E70
:1023B000DBCF25F0A5EC2EF0195002019E25276EEB
:1023C0001A509F21286E1B50A021296E1C50A1215C
:1023D0002A6ECAC21DF0CBC21EF0CCC21FF0CDC205
:1023E00020F0BAC222F0BBC223F0BCC224F0BDC2AE
:1023F00025F0A5EC2EF01950275C0201B26F1A509F
:102400002858B36F1B502958B46F1C502A58B56F09
:10241000B2C21DF0B3C21EF0B4C21FF0B5C220F0AC
:10242000BEC222F0BFC223F0C0C224F0C1C225F058
:1024300060EC2FF01DC0CEF21EC0CFF21FC0D0F254
:1024400020C0D1F2CEC21DF0CFC21EF0D0C21FF00C
:10245000D1C220F0BEC222F0BFC223F0C0C224F01D
:10246000C1C225F0A5EC2EF019500201B25DDA6F61
:102470001A50B359DB6F1B50B459DC6F1C50B5595F
:10248000DD6FD9CFE9FFDACFEAFFEE50CE5DEE5037
:10249000CF59EE50D059EE50D1593DE2DAC21DF07D
:1024A000DBC21EF0DCC21FF0DDC220F0DFCF22F065
:1024B000010EDBCF23F0020EDBCF24F0030EDBCFC7
:1024C00025F0A5EC2EF019500201A225276E1A5016
:1024D000A321286E1B50A421296E1C50A5212A6E11
:1024E000CEC21DF0CFC21EF0D0C21FF0D1C220F06C
:1024F000C2C222F0C3C223F0C4C224F0C5C225F078
:10250000A5EC2EF01950275C1A5028581B5029585A
:102510001C502A5824E20201CE07000ECF5BD05B8C
:10252000D15BBE0EE96E020EEA6EDA51EE24DA6F6E
:10253000DB51EE20DB6FDC51EE20DC6FDD51EE2055
:10254000DD6FD9CFE9FFDACFEAFFEE50DA5DEE506A
:10255000DB59EE50DC59EE50DD5901E292D7020111
:10256000D651D711D811D91122E0CAC21DF0CBC261
:102570001EF0CCC21FF0CDC220F0DFCF22F0010E42
:10258000DBCF23F0020EDBCF24F0030EDBCF25F0F0
:10259000A5EC2EF019500201CE25D66F1A50CF218E
:1025A000D76F1B50D021D86F1C50D121D96FD26B5F
:1025B000D36BD46BD56B100E1F0BCAC2D2F2CBC239
:1025C000D3F2CCC2D4F2CDC2D5F208E00201D89049
:1025D000D237D337D437D537E806F9E10201D26BC9
:1025E000D36BCEC227F0CFC228F0D0C229F0D1C21F
:1025F0002AF0296A2A6AD20EE96E020EEA6EEE50BD
:102600002710D26FEE502810D36FEE502910D46FE0
:10261000EE502A10D56F060EE15C02E2E16AE55247
:10262000E16EE552E7CFD9FF1200D9CFE6FFE1CF47
:10263000D9FF020EE126FB0EDBCF27F0FC0EDBCF2D
:1026400028F0FD0EDBCF29F0FE0EDBCF2AF027505D
:10265000281029102A1004E1200EF36EF46A1FD10D
:10266000DE6ADD6AD950FB0FE96EFF0EDA20EA6EF2
:10267000D880FF0EEE54FF0EEE54000EEE54000E06
:10268000EE542EE3DECF27F0DDCF28F0100E272604
:10269000000E282227C0DEFF28C0DDFFFB0EDBCFA7
:1026A00027F0FC0EDBCF28F0FD0EDBCF29F0FE0E6D
:1026B000DBCF2AF0100E1F0B07E0D8902736283604
:1026C00029362A36E806F9E1FB0E27C0DBFFFC0EAF
:1026D00028C0DBFFFD0E29C0DBFFFE0E2AC0DBFF9A
:1026E000D950FB0FE96EFF0EDA20EA6ED880FF0E9C
:1026F000EE54FF0EEE54FF0EEE54000EEE542EE399
:10270000DECF27F0DDCF28F0080E2726000E282286
:1027100027C0DEFF28C0DDFFFB0EDBCF27F0FC0E5D
:10272000DBCF28F0FD0EDBCF29F0FE0EDBCF2AF049
:10273000080E1F0B07E0D8902736283629362A3690
:10274000E806F9E1FB0E27C0DBFFFC0E28C0DBFF2B
:10275000FD0E29C0DBFFFE0E2AC0DBFFD950FB0FA8
:10276000E96EFF0EDA20EA6ED880FF0EEE54FF0EFF
:10277000EE54FF0EEE540F0EEE542EE3DECF27F094
:10278000DDCF28F0040E2726000E282227C0DEFF0A
:1027900028C0DDFFFB0EDBCF27F0FC0EDBCF28F0DF
:1027A000FD0EDBCF29F0FE0EDBCF2AF0040E1F0B4F
:1027B00007E0D8902736283629362A36E806F9E188
:1027C000FB0E27C0DBFFFC0E28C0DBFFFD0E29C07F
:1027D000DBFFFE0E2AC0DBFFD950FB0FE96EFF0EB8
:1027E000DA20EA6ED880FF0EEE54FF0EEE54FF0E94
:1027F000EE543F0EEE542EE3DECF27F0DDCF28F06F
:10280000020E2726000E282227C0DEFF28C0DDFF8B
:10281000FB0EDBCF27F0FC0EDBCF28F0FD0EDBCF6D
:1028200029F0FE0EDBCF2AF0020E1F0B07E0D89036
:102830002736283629362A36E806F9E1FB0E27C066
:10284000DBFFFC0E28C0DBFFFD0E29C0DBFFFE0E08
:102850002AC0DBFFD950FB0FE96EFF0EDA20EA6ECB
:10286000D880FF0EEE54FF0EEE54FF0EEE547F0E96
:10287000EE540CE3DECF27F0DDCF28F0010E272643
:10288000000E282227C0DEFF28C0DDFFDECF27F0A4
:10289000DDCF28F027C0F3FF28C0F4FF00D0020EE0
:1028A000E15C02E2E16AE552E16EE552E7CFD9FF71
:1028B0001200D9CFE6FFE1CFD9FF200EE126C0C23A
:1028C00027F0C1C228F00001296A2A6A296A2A6A07
:1028D000100E27C0DBFF110E28C0DBFF120E29C02F
:1028E000DBFF130E2AC0DBFFBEC227F0BFC228F0F9
:1028F000C0C229F0C1C22AF0296A2A6A140E27C070
:10290000DBFF150E28C0DBFF160E29C0DBFF170EFC
:102910002AC0DBFFC4C227F0C5C228F0296A2A6A90
:10292000296A2A6A180E27C0DBFF190E28C0DBFFB0
:102930001A0E29C0DBFF1B0E2AC0DBFFC2C227F024
:10294000C3C228F0C4C229F0C5C22AF0296A2A6A83
:102950001C0E27C0DBFF1D0E28C0DBFF1E0E29C08A
:10296000DBFF1F0E2AC0DBFF140EDBCF27F0150E96
:10297000DBCF28F0160EDBCF29F0170EDBCF2AF0C5
:1029800027C01DF028C01EF029C01FF02AC020F06B
:102990001C0EDBCF22F01D0EDBCF23F01E0EDBCF93
:1029A00024F01F0EDBCF25F0A5EC2EF0040E19C08D
:1029B000DBFF050E1AC0DBFF060E1BC0DBFF070E98
:1029C0001CC0DBFF100EDBCF2FF0110EDBCF30F081
:1029D000120EDBCF31F0130EDBCF32F02FC01DF023
:1029E00030C01EF031C01FF032C020F01C0EDBCF13
:1029F00022F01D0EDBCF23F01E0EDBCF24F01F0EC6
:102A0000DBCF25F0A5EC2EF019C02BF01AC02CF06E
:102A10001BC02DF01CC02EF0180EDBCF33F0190EAA
:102A2000DBCF34F01A0EDBCF35F01B0EDBCF36F0E8
:102A300033C01DF034C01EF035C01FF036C020F08A
:102A4000140EDBCF22F0150EDBCF23F0160EDBCFFA
:102A500024F0170EDBCF25F0A5EC2EF02B50192417
:102A6000276E2C501A20286E2D501B20296E2E50B8
:102A70001C202A6E080E27C0DBFF090E28C0DBFFD2
:102A80000A0E29C0DBFF0B0E2AC0DBFF040EDBCFD2
:102A90002FF0050EDBCF30F0060EDBCF31F0070E46
:102AA000DBCF32F031C02BF032C02CF000012D6AA8
:102AB0002E6A2D6A2E6AD950080FE96EDACFEAFF26
:102AC0002B50EE24276E2C50EE20286E2D50EE2039
:102AD000296E2E50EE202A6E0C0E27C0DBFF0D0E45
:102AE00028C0DBFF0E0E29C0DBFF0F0E2AC0DBFF64
:102AF00027682868296A2A6AD950040FE96EDACF54
:102B0000EAFFEE502716EE502816EE502916EE502A
:102B10002A162B682C682D6A2E6AD9500C0FE96E84
:102B2000DACFEAFFEE502B16EE502C16EE502D1693
:102B3000EE502E16100E1F0B07E0D8902B362C36B9
:102B40002D362E36E806F9E12B5027122C5028128C
:102B50002D5029122E502A12040E27C0DBFF050E1D
:102B600028C0DBFF060E29C0DBFF070E2AC0DBFFF3
:102B70000C0EDBCF2BF00D0EDBCF2CF00E0EDBCFCF
:102B80002DF00F0EDBCF2EF02DC027F02EC028F039
:102B90000001296A2A6A296A2A6A27C0DFFF010E12
:102BA00028C0DBFF020E29C0DBFF030E2AC0DBFFBB
:102BB000100EDBCF2BF0110EDBCF2CF0120EDBCF83
:102BC0002DF0130EDBCF2EF02BC01DF02CC01EF00D
:102BD0002DC01FF02EC020F0180EDBCF22F0190EF2
:102BE000DBCF23F01A0EDBCF24F01B0EDBCF25F05A
:102BF000A5EC2EF019C027F01AC028F01BC029F050
:102C00001CC02AF02750DE262850DE222950DE2262
:102C10002A50DD22DD52DD52DFCFA6F2010EDBCFDE
:102C2000A7F2020EDBCFA8F2030EDBCFA9F2040E4F
:102C3000DBCFAAF2050EDBCFABF2060EDBCFACF298
:102C4000070EDBCFADF2200EE15C02E2E16AE55255
:102C5000E16EE552E7CFD9FF12009EEC21F046C2AB
:102C60004AF247C24BF248C24CF249C24DF24A0EF8
:102C7000E66E020EE66E070EE66EF8EC0DF0E5521B
:102C8000E552E55234D84AC246F24BC247F24CC232
:102C900048F24DC249F2E66AE8C2E6FF020EE66E6D
:102CA00009EC21F0E552E552E55212001F0E020137
:102CB0000015856F070E0115866F8651200DF3CF25
:102CC0008CF2E00E8C1785518C130C0E8A6F46EC3B
:102CD0000DF00DD885C223F286C222F20201AA0E9F
:102CE000216F550E206F04C224F267EF0CF085C2ED
:102CF00027F0286A296A2A6A4AC21DF04BC21EF0D0
:102D00004CC21FF04DC220F027C022F028C023F093
:102D100029C024F02AC025F0A5EC2EF019C04EF2EF
:102D20001AC04FF21BC050F21CC051F202019C515C
:102D300009E0A669A769A869A96BAA6BAB6BAC6B24
:102D4000AD6909D0A669A7690F0EA86FA96BAA6B18
:102D5000AB6BAC6BAD694EC2BAF24FC2BBF250C2A4
:102D6000BCF251C2BDF243EC10F0D2C252F2D3C257
:102D700053F2D4C254F2D5C255F2520EE66E020E90
:102D8000E66E100EE66EF8EC0DF0E552E552E552F7
:102D9000CAEF16F0D9CFE6FFE1CFD9FF060EE12644
:102DA000165005E102019751DE6EDD6A05D0020181
:102DB00097390F0BDE6EDD6A0F0EDE16DD6A000E30
:102DC000DFCF1FF0010EDBCF20F0050E1F1801E151
:102DD000205039E0040E1F1801E120502BE0030EB3
:102DE0001F1801E120501DE0020E1F1801E12050C4
:102DF0000FE0010E1F1801E1205001E025D06AC24A
:102E00005AF26BC25BF26CC25CF26DC25DF224D00E
:102E10006EC25AF26FC25BF270C25CF271C25DF2B6
:102E20001BD072C25AF273C25BF274C25CF275C2FA
:102E30005DF212D076C25AF277C25BF278C25CF2CF
:102E400079C25DF209D008D076C25AF277C25BF23D
:102E500078C25CF279C25DF2020E5AC2DBFF030E49
:102E60005BC2DBFF040E5CC2DBFF050E5DC2DBFF55
:102E7000165001E0F3D00F0E9615DE6EDD6AD9CF45
:102E8000E9FFDACFEAFFEE50ED1001E193D0000E3A
:102E9000DFCF1FF0010EDBCF20F0030E1F1801E182
:102EA000205052E0020E1F1801E1205023E0010ED5
:102EB0001F1801E1205001E071D0620EE96E020E90
:102EC000EA6E5A51EE24276E5B51EE20286E5C515B
:102ED000EE20296E5D51EE202A6E020E27C0DBFF28
:102EE000030E28C0DBFF040E29C0DBFF050E2AC03D
:102EF000DBFF60D05A0EE96E020EEA6EEE50625DA4
:102F0000EE506359EE506459EE5065591CE2620E62
:102F1000E96E020EEA6EEE505A5D276EEE505B5976
:102F2000286EEE505C59296EEE505D592A6E020EE5
:102F300027C0DBFF030E28C0DBFF040E29C0DBFF28
:102F4000050E2AC0DBFF36D0620EE96E020EEA6E75
:102F5000EE505A5DEE505B59EE505C59EE505D59A3
:102F60001CE25A0EE96E020EEA6EEE50625D276EAA
:102F7000EE506359286EEE506459296EEE50655933
:102F80002A6E020E27C0DBFF030E28C0DBFF040EF3
:102F900029C0DBFF050E2AC0DBFF0CD0020E5AC28F
:102FA000DBFF030E5BC2DBFF040E5CC2DBFF050E22
:102FB0005DC2DBFF00017D5150E0000E0201E21511
:102FC000276E800EE315286E275002E1800E281828
:102FD00025E1E39FE2C22BF0E3C22CF02D6A2E6ABA
:102FE000D950020FE96EDACFEAFF2B50EE5C276E64
:102FF0002C50EE58286E2D50EE58296E2E50EE585B
:103000002A6E020E27C0DBFF030E28C0DBFF040E72
:1030100029C0DBFF050E2AC0DBFF1FD0E2C227F06C
:10302000E3C228F0296A2A6AD950020FE96EDACF82
:10303000EAFFEE502726EE502822EE502922EE50CD
:103040002A22020E27C0DBFF030E28C0DBFF040E7E
:1030500029C0DBFF050E2AC0DBFFB2D0F00E9615AB
:10306000DE6EDD6AD9CFE9FFDACFEAFF040E0F0B7F
:1030700006E0EC52D890ED32EF32E806FAE10F0E9E
:10308000DE16DD6AD9CFE9FFDACFEAFFEE50ED10A8
:1030900001E196D0000EDFCF1FF0010EDBCF20F054
:1030A000030E1F1801E1205054E0020E1F1801E129
:1030B000205024E0010E1F1801E1205001E074D0DF
:1030C000660EE96E020EEA6E02015A51EE24276E78
:1030D0005B51EE20286E5C51EE20296E5D51EE2092
:1030E0002A6E020E27C0DBFF030E28C0DBFF040E92
:1030F00029C0DBFF050E2AC0DBFF62D05A0EE96E45
:10310000020EEA6EEE500201665DEE506759EE5017
:103110006859EE5069591CE2660EE96E020EEA6EBD
:10312000EE505A5D276EEE505B59286EEE505C599A
:10313000296EEE505D592A6E020E27C0DBFF030E8A
:1031400028C0DBFF040E29C0DBFF050E2AC0DBFF11
:1031500037D0660EE96E020EEA6EEE5002015A5D3D
:10316000EE505B59EE505C59EE505D591CE25A0E20
:10317000E96E020EEA6EEE50665D276EEE506759FC
:10318000286EEE506859296EEE5069592A6E020E6B
:1031900027C0DBFF030E28C0DBFF040E29C0DBFFC6
:1031A000050E2AC0DBFF0CD0020E5AC2DBFF030E55
:1031B0005BC2DBFF040E5CC2DBFF050E5DC2DBFF02
:1031C00086C227F0286A296A2A6A27C01DF028C00B
:1031D0001EF029C01FF02AC020F0020EDBCF22F023
:1031E000030EDBCF23F0040EDBCF24F0050EDBCF84
:1031F00025F0A5EC2EF019C056F21AC057F21BC0EC
:1032000058F21CC059F256C2BEF257C2BFF258C2A1
:10321000C0F259C2C1F252C2C2F253C2C3F254C286
:10322000C4F255C2C5F259EC14F0080E1F0BA6C229
:103230005EF2A7C25FF2A8C260F2A9C261F208E022
:103240000201D8905E375F3760376137E806F9E1F1
:1032500002015E6B180E1F0BAAC227F0ABC228F04A
:10326000ACC229F0ADC22AF007E0D8902A32293248
:1032700028322732E806F9E1286A296A2A6A5E0EAE
:10328000E96E020EEA6EEE50271002015E6FEE50FC
:1032900028105F6FEE502910606FEE502A10616F9A
:1032A000885159E0020E5EC2DBFF030E5FC2DBFFF6
:1032B000040E60C2DBFF050E61C2DBFF030EDE6E93
:1032C000DD6ADECF27F0DDCF28F00001800E281464
:1032D00040E12768286A296A2A6AD950020FE96EF4
:1032E000DACFEAFFEE502716EE502816EE502916D8
:1032F000EE502A16DECFE9FFDDCFEAFFE40EE92625
:10330000020EEA2227C0EFFF020EDBCF27F0030EEA
:10331000DBCF28F0040EDBCF29F0050EDBCF2AF03F
:10332000080ED8902A32293228322732E806F9E1ED
:10333000020E27C0DBFF030E28C0DBFF040E29C0EE
:10334000DBFF050E2AC0DBFFDF06010E01E2DB0614
:10335000B8D737EC08F00201940501E10AD8060E4F
:10336000E15C02E2E16AE552E16EE552E7CFD9FFA6
:103370001200D9CFE6FFE1CFD9FF0C0EE126080EEF
:10338000DB68030EF36E090EF3CFDBFF060EDB6A7C
:10339000070EDB6A0101220EF86F5E0EF96F5AC24A
:1033A00027F05BC228F05CC229F05DC22AF00C0E47
:1033B000D8902A32293228322732E806F9E1040E61
:1033C00027C0DBFF050E28C0DBFFF8C1F6FFF9C1FF
:1033D000F7FF08000A0EF5CFDBFF010EF36E060EB5
:1033E000F3CFDBFF070EDB6A0B0EDB6A0A0EDB5046
:1033F000F36E0B0EDBCFF4FFF350F45C01E38CD0E3
:10340000060EDBCF27F0DB2A070EDBCF28F001E327
:10341000DB2A010ED89027362836E806FBE10101A9
:10342000F8512724F66EF9512820F76E0900F5CFE0
:10343000DEFF0A00F5CFDDFF060EDBCF27F0DB2A2B
:10344000070EDBCF28F001E3DB2A010ED8902736E8
:103450002836E806FBE10101F8512724F66EF95100
:103460002820F76E0900020EF5CFDBFF0A00030EDD
:10347000F5CFDBFFD9CFE9FFDACFEAFFEE50ED1051
:1034800011E1D950020FE96EDACFEAFFFF0EEE1814
:1034900002E1FF0EED1806E10B0EDB50E76E090EA0
:1034A000E7CFDBFFDECF27F0DDCF28F0040EDBCF48
:1034B00029F0050EDBCF2AF02750295C28502A5826
:1034C00028E3040EDBCF2BF0050EDBCF2CF0020E31
:1034D000DBCF2DF0030EDBCF2EF02B502D5C2C50CC
:1034E0002E5817E3090EDB50F36E0B0EDB50F35C26
:1034F00010E0DECFDEF2DDCFDFF2020EDBCFE0F256
:10350000030EDBCFE1F20B0EDB50E76E080EE7CFC8
:10351000DBFF0B0EDB2A6AD7080EDB50FF0806E143
:10352000090EDB50E76E080EE7CFDBFF080EDB501D
:103530000201955D07E0080EDBCFE4F2010EE56FB6
:10354000D2EC0FF00C0EE15C02E2E16AE552E16EB2
:10355000E552E7CFD9FF1200D9CFE6FFE1CFD9FF7F
:10356000E652E4C2DFFF000EDF90DF92DF94DF96C9
:10357000DF9E0201010E846FDF50700A01E14ED11F
:10358000200A01E113D1100A01E1CDD0700A01E156
:1035900093D0100A5AE0300A17E0100A01E08BD1EC
:1035A0004AC246F24BC247F24CC248F24DC249F2FF
:1035B000DFCFE6FF04C2E6FF020EE66E09EC21F063
:1035C000E552E552E55281D19D5134E1010E9D6FE6
:1035D0004AC27AF24BC27BF24CC27CF24DC27DF2FF
:1035E00072C27EF273C27FF274C280F275C281F23F
:1035F00097C283F2330E976F86C282F2800EE41573
:10360000800802E0010E866F77EC16F072C246F277
:1036100073C247F274C248F275C249F2DFCFE6FFC7
:1036200004C2E6FF020EE66E09EC21F0E552E55217
:10363000E5520AD0E66A04C2E6FF040EE66E09EC23
:1036400021F0E552E552E55240D19D512AE09EEC31
:1036500021F00F0E02014917460EE96E020EEA6EC6
:103660004A51EE244A6F4B51EE204B6F4C51EE20E5
:103670004C6F4D51EE204D6F77EC16F04AC246F27A
:103680004BC247F24CC248F24DC249F2E66A04C24C
:10369000E6FF020EE66E09EC21F0E552E552E55236
:1036A0000AD0E66A04C2E6FF040EE66E09EC21F0D9
:1036B000E552E552E55209D19D512AE09EEC21F0F8
:1036C0000F0E02014917460EE96E020EEA6EEE5029
:1036D0004A5D4A6FEE504B594B6FEE504C594C6F50
:1036E000EE504D594D6F77EC16F04AC246F24BC280
:1036F00047F24CC248F24DC249F2E66A04C2E6FF04
:10370000020EE66E09EC21F0E552E552E5520AD0D0
:10371000E66A04C2E6FF040EE66E09EC21F0E5520B
:10372000E552E552D2D09D5136E09D6B7EC272F2D9
:103730007FC273F280C274F281C275F283C297F2C3
:1037400082C286F24AC27AF24BC27BF24CC27CF24F
:103750004DC27DF27A0EE66E020EE66E070EE66E42
:10376000F8EC0DF0E552E552E55277EC16F04AC25E
:1037700046F24BC247F24CC248F24DC249F2DFCF8B
:10378000E6FF04C2E6FF020EE66E09EC21F0E55208
:10379000E552E5520AD0E66A04C2E6FF040EE66E80
:1037A00009EC21F0E552E552E5528FD09D512BE016
:1037B0009D6B7AC24AF27BC24BF27CC24CF27DC254
:1037C0004DF27EC272F27FC273F280C274F281C285
:1037D00075F283C297F282C286F277EC16F04AC283
:1037E00046F24BC247F24CC248F24DC249F2DFCF1B
:1037F000E6FF04C2E6FF020EE66E09EC21F0E55298
:10380000E552E5520AD0E66A04C2E6FF040EE66E0F
:1038100009EC21F0E552E552E55257D09D5140E1C7
:10382000010E9D6F4AC27AF24BC27BF24CC27CF20F
:103830004DC27DF297C283F2330E976F9EEC21F05A
:103840000F0E0201491772C27EF273C27FF274C278
:1038500080F275C281F246C272F247C273F248C268
:1038600074F249C275F286C282F2800EE4158008B5
:1038700002E0010E866F77EC16F05AC246F25BC288
:1038800047F25CC248F25DC249F2E66A04C2E6FF52
:10389000020EE66E09EC21F0E552E552E5520AD03F
:1038A000E66A04C2E6FF040EE66E09EC21F0E5527A
:1038B000E552E5520AD0E66A04C2E6FF010EE66E62
:1038C00009EC21F0E552E552E552E552E552E7CF29
:1038D000D9FF1200D9CFE6FFE1CFD9FF090EE126CB
:1038E000DE6ADE6ADE6ADD6ADD52DD520201005107
:1038F000140A01E172D2070A01E111D2010A01E1C1
:10390000D8D1030A01E186D1010A01E12CD11F0AB5
:1039100001E11DD1010A01E10ED1030A01E1FFD04D
:10392000010A01E1F0D0070A01E1E1D0010A01E159
:10393000D2D0030A01E1C3D0010A63E00F0A55E0C7
:10394000010A47E0030A39E0010A2BE0070A1DE0FB
:10395000010A0FE0030A01E0CED24AC2DFFF010EE6
:103960004BC2DBFF020E4CC2DBFF030E4DC2DBFF7E
:10397000CCD24EC2DFFF010E4FC2DBFF020E50C29F
:10398000DBFF030E51C2DBFFC0D256C2DFFF010EC8
:1039900057C2DBFF020E58C2DBFF030E59C2DBFF2A
:1039A000B4D25AC2DFFF010E5BC2DBFF020E5CC263
:1039B000DBFF030E5DC2DBFFA8D25EC2DFFF010E9C
:1039C0005FC2DBFF020E60C2DBFF030E61C2DBFFE2
:1039D0009CD246C2DFFF010E47C2DBFF020E48C287
:1039E000DBFF030E49C2DBFF90D242C2DFFF010EB4
:1039F00043C2DBFF020E44C2DBFF030E45C2DBFF06
:103A000084D2000E96C2DFFF010EDB6A020EDB6A73
:103A1000030EDB6AD9CFE9FFDACFEAFFEF50EE6A97
:103A2000EFCFF4FFEE6EEF50F4CFEEFFEF6E88C2F3
:103A300027F0286A296A2A6A2750DE122850DE12E7
:103A40002950DE122A50DD12DD52DD52D9CFE9FFB6
:103A5000DACFEAFFEF50EE6AEFCFF4FFEE6EEF50F1
:103A6000F4CFEEFFEF6E86C227F0286A296A2A6A31
:103A70002750DE122850DE122950DE122A50DD12A5
:103A8000DD52DD52D9CFE9FFDACFEAFFEF50EE6A1F
:103A9000EFCFF4FFEE6EEF50F4CFEEFFEF6E85C286
:103AA00027F0286A296A2A6A2750DE122850DE1277
:103AB0002950DE122A50DD12DD52DD5226D252C2CA
:103AC000DFFF010E53C2DBFF020E54C2DBFF030E09
:103AD00055C2DBFF1AD262C2DFFF010E63C2DBFFF9
:103AE000020E64C2DBFF030E65C2DBFF0ED266C2AC
:103AF000DFFF010E67C2DBFF020E68C2DBFF030EB1
:103B000069C2DBFF02D26AC2DFFF010E6BC2DBFFBC
:103B1000020E6CC2DBFF030E6DC2DBFFF6D16EC27C
:103B2000DFFF010E6FC2DBFF020E70C2DBFF030E70
:103B300071C2DBFFEAD172C2DFFF010E73C2DBFF8D
:103B4000020E74C2DBFF030E75C2DBFFDED176C24C
:103B5000DFFF010E77C2DBFF020E78C2DBFF030E30
:103B600079C2DBFFD2D1000EDEC2DFFF010EDFC261
:103B7000DBFF020EDB6A030EDB6AD9CFE9FFDACF87
:103B8000EAFFEECF27F0EECF28F0EECF29F0EFCF0F
:103B90002AF0100E1F0B07E0D8902736283629365A
:103BA0002A36E806F9E127C0DFFF010E28C0DBFF57
:103BB000020E29C0DBFF030E2AC0DBFF276A286A3A
:103BC00029682A68D9CFE9FFDACFEAFFEE50271635
:103BD000EE502816EE502916EE502A1627C0DFFFA9
:103BE000010E28C0DBFF020E29C0DBFF030E2AC036
:103BF000DBFFE0C227F0E1C228F0296A2A6A2750D9
:103C0000DE122850DE122950DE122A50DD12DD525B
:103C1000DD527BD1000E97C2DFFF010EDB6A020E80
:103C2000DB6A030EDB6AD9CFE9FFDACFEAFFEF5098
:103C3000EE6AEFCFF4FFEE6EEF50F4CFEEFFEF6ED3
:103C400094C227F0286A296A2A6A2750DE1228506F
:103C5000DE122950DE122A50DD12DD52DD52D9CF9C
:103C6000E9FFDACFEAFFEF50EE6AEFCFF4FFEE6E36
:103C7000EF50F4CFEEFFEF6E95C227F0286A296A65
:103C80002A6A2750DE122850DE122950DE122A50EE
:103C9000DD12DD52DD52D9CFE9FFDACFEAFFEF5076
:103CA000EE6AEFCFF4FFEE6EEF50F4CFEEFFEF6E63
:103CB0002CD17DC027F0286A296A2A6A27AE03D052
:103CC000286829682A6827C0DFFF010E28C0DBFFAB
:103CD000020E29C0DBFF030E2AC0DBFFD9CFE9FFAC
:103CE000DACFEAFF100EE76ED890EF36010EEB3612
:103CF000020EEB36030EEB36E706F6E1E2C227F0E2
:103D0000E3C228F0296A2A6A2750DE122850DE1200
:103D10002950DE122A50DD12DD52DD52F6D0000E9F
:103D200089C2DFFF010EDB6A020EDB6A030EDB6A6B
:103D3000D9CFE9FFDACFEAFFEF50EE6AEFCFF4FF19
:103D4000EE6EEF50F4CFEEFFEF6E0450276E286A50
:103D5000296A2A6A2750DE122850DE122950DE1204
:103D60002A50DD12DD52DD52D9CFE9FFDACFEAFF6A
:103D7000EF50EE6AEFCFF4FFEE6EEF50F4CFEEFFB0
:103D8000EF6E0550276E286A296A2A6A2750DE12CC
:103D90002850DE122950DE122A50DD12DD52DD528B
:103DA000D9CFE9FFDACFEAFFEF50EE6AEFCFF4FFA9
:103DB000EE6EEF50F4CFEEFFEF6E99C227F0286A57
:103DC000296A2A6A2750DE122850DE122950DE1294
:103DD0002A50DD12DD52DD5298D00151020A1CE05A
:103DE000030A01E06FD0060EE7C2DBFFDB50040DD3
:103DF000F3CFE9FFF4CFEAFF420EE926010EEA22F3
:103E0000EECFDFFF010EEECFDBFF020EEECFDBFFCA
:103E1000030EEECFDBFF6ED0060EE7C2DBFFDB2A20
:103E2000DBCFE7FFE79EE746E7CFDBFFDBCFF3FF24
:103E3000DB2AF350E96EEA6AD890E936EA36000EDA
:103E4000E926010EEA22EECF27F0EFCF28F0000E90
:103E500027C0DFFF010E28C0DBFF020EDB6A030E66
:103E6000DB6AD9CFE9FFDACFEAFF100EE76ED89010
:103E7000EF36010EEB36020EEB36030EEB36E7069D
:103E8000F6E1D9CFE9FFDACFEAFFEE6AEE6A060E75
:103E9000EA6ADB34FE0BEA36E96E000EE926010E13
:103EA000EA22EECF27F0EFCF28F0296A2A6A2750BE
:103EB000DE122850DE122950DE122A50DD12DD52A9
:103EC000DD5218D0060EE7C2DBFFDB50040DF3CF46
:103ED000E9FFF4CFEAFF720EE926010EEA22EECFE7
:103EE000DFFF010EEECFDBFF020EEECFDBFF030E96
:103EF000EECFDBFF0AD0040EDE6E030EDE6E020E86
:103F0000DE6E010EDD6EDD52DD52DFCF46F2010EB8
:103F1000DBCF47F2020EDBCF48F2030EDBCF49F2D4
:103F2000E66A00C2E6FF020EE66E73D9E552E5527C
:103F3000E552090EE15C02E2E16AE552E16EE5520A
:103F4000E7CFD9FF1200D9CFE6FFE1CFD9FF050EA9
:103F5000E126030EDB6A040EDB6AE4C2DFFF000E1B
:103F6000DF90DF92DF94DF96DF98E8D91F0E020121
:103F70004917010EDB6A020EDB6ADF50A00A01E17D
:103F800005D1400A01E1ABD0200A4EE0400A43E0EF
:103F9000E00A2DE0200A17E0600A01E019D146C2CC
:103FA0006AF247C26BF248C26CF249C26DF26A0E05
:103FB000E66E020EE66E4A0EE66EF8EC0DF0E55285
:103FC000E552E5520FD146C26EF247C26FF248C2C7
:103FD00070F249C271F26E0EE66E020EE66E4E0E81
:103FE000E66EF8EC0DF0E552E552E552FBD046C224
:103FF00072F247C273F248C274F249C275F2720E8D
:10400000E66E020EE66E520EE66EF8EC0DF0E5522C
:10401000E552E552E7D046C276F247C277F248C28F
:1040200078F249C279F2DED046C262F247C263F248
:1040300048C264F249C265F2070E6517180EE4150E
:10404000276E286A27BE2868010E27C0DBFF020EF4
:1040500028C0DBFFD950010FE96EDACFEAFF0F0E5F
:10406000EE1801E1ED5035E0010EDBCF27F0020E36
:10407000DBCF28F0030ED89028322732E804FBE18A
:10408000010E27C0DBFF020E28C0DBFF030EE76E28
:10409000010EDBCF27F0020EDBCF28F0E75027160A
:1040A000286A010E27C0DBFF020E28C0DBFFF00EDE
:1040B00002019615966F9651296E2A6A010EDB5001
:1040C0002910276E020EDB502A10286E27C096F2A8
:1040D00003D0F00E9615966F165000E183D046C2BD
:1040E00066F247C267F248C268F249C269F2070E37
:1040F0006917180EE415276E286A27BE2868010E76
:1041000027C0DBFF020E28C0DBFFD950010FE96E8C
:10411000DACFEAFF0F0EEE1801E1ED5031E0010EAB
:10412000DBCF27F0020EDBCF28F0D89027362836D9
:10413000010E27C0DBFF020E28C0DBFF300EE76E4A
:10414000010EDBCF27F0020EDBCF28F0E750271659
:10415000286A010E27C0DBFF020E28C0DBFF0F0E0E
:104160009615966F9651296E2A6A010EDB5029101A
:10417000276E020EDB502A10286E27C096F203D05D
:104180000F0E9615966F165000E12CD0040E1F0BE3
:1041900008E00201D8904637473748374937E806E4
:1041A000F9E1F00E0201461746C242F247C243F25D
:1041B00048C244F249C245F2420EE66E020EE66E75
:1041C0001C0EE66EF8EC0DF0E552E552E5520AD011
:1041D000DFCFE6FF770EE66E040EE66E1AD8E552E4
:1041E000E552E552165002E1CAEC16F0E66A770E87
:1041F000E66E010EE66E0DD8E552E552E552050E6B
:10420000E15C02E2E16AE552E16EE552E7CFD9FFF7
:104210001200D9CFE6FFE1CFD9FF060EE126FE0E50
:10422000DB50030A74E0010A12E0030A07E0E4C26B
:1042300020F2020121692269236971D000C220F2B3
:1042400001C221F202C222F203C223F268D046C2A6
:10425000DFFF010E47C2DBFF020E48C2DBFF030E89
:1042600049C2DBFFF36E040EF3CFDBFF050EDB6A02
:10427000040EDBCF27F0050EDBCF28F00001800E07
:10428000281440E1D9CFE9FFDACFEAFFEECF27F0DB
:10429000EECF28F0EECF29F0EFCF2AF02750E66ED0
:1042A000040EDBCFE9FF050EDBCFEAFF200EE92687
:1042B000020EEA22E552E750EF6ED9CFE9FFDACFDE
:1042C000EAFFEECF27F0EECF28F0EECF29F0EFCFC8
:1042D0002AF0080ED8902A32293228322732E806EE
:1042E000F9E127C0DFFF010E28C0DBFF020E29C065
:1042F000DBFF030E2AC0DBFF040EDB06050E01E226
:10430000DB06B6D7FC0EDB500201201308D0FC0EF2
:10431000DBCF20F20201216B226B236B00D0FD0E5C
:10432000DBCF24F267EC0CF0060EE15C02E2E16AFE
:10433000E552E16EE552E7CFD9FF1200D9CFE6FF93
:10434000E1CFD9FF040EE1260201466B476B486BB3
:10435000496BDE6ADD6ADECF27F0DDCF28F0D8902A
:10436000285004E6040E275C000E28584DE2080E83
:104370001F0B08E00201D8904637473748374937C6
:10438000E806F9E1DECFE9FFDDCFEAFFE40EE9263A
:10439000020EEA22EFCF27F0286A27BE2868020E15
:1043A00027C0DBFF030E28C0DBFFFF0EE76E020E07
:1043B000DBCF27F0030EDBCF28F0E7502716286A63
:1043C000020E27C0DBFF030E28C0DBFF020EDBCF8F
:1043D00027F0030EDBCF28F0296A2A6A460EE96E21
:1043E000020EEA6EEE5027100201466FEE502810C2
:1043F000476FEE502910486FEE502A10496FDF2AA0
:10440000010E01E3DB2AA7D7040EE15C02E2E16AB8
:10441000E552E16EE552E7CFD9FF1200D9CFE6FFB2
:10442000E1CFD9FF090EE126010EDB6A020EDB6A3D
:10443000010EDB6A800E0201E415800806E1010E20
:10444000F36E020EF3CFDBFF02D0020EDB6A7F0EAB
:10445000E415DF6EDF5001E197D27F0EE415DF6EC9
:10446000DF50140A01E18FD2070A01E18BD2010A61
:1044700001E187D2030A01E181D2010A01E147D2B9
:104480001C0A01E123D2070A01E1E6D1010A01E198
:1044900088D1030A01E152D1010A01E12AD10E0AB1
:1044A00001E1CCD0030A01E196D0010A6FE0070ACE
:1044B00033E0010A1AE0030A01E066D26AC26EF232
:1044C0006BC26FF26CC270F26DC271F2020EDB5001
:1044D0000BE06E0EE66E020EE66E4E0EE66EF8EC29
:1044E0000DF0E552E552E5524FD26EC26AF26FC24C
:1044F0006BF270C26CF271C26DF2020EDB500BE017
:104500006A0EE66E020EE66E4A0EE66EF8EC0DF0EE
:10451000E552E552E55238D2030E6AC2DBFF040EC3
:104520006BC2DBFF050E6CC2DBFF060E6DC2DBFF4C
:104530006EC26AF26FC26BF270C26CF271C26DF23F
:10454000030EDBCF6EF2040EDBCF6FF2050EDBCF76
:1045500070F2060EDBCF71F2020EDB500BE06A0E3A
:10456000E66E020EE66E4A0EE66EF8EC0DF0E552CF
:10457000E552E5526E0EE66E020EE66E4E0EE66EE9
:10458000F8EC0DF0E552E552E552FED10F0EE615BE
:10459000276E286A27BE2868070E27C0DBFF080E93
:1045A00028C0DBFF070EDBCFE9FF080EDBCFEAFFF9
:1045B000D890E936EA36D890E936EA36720EE9261E
:1045C000010EEA226AC2EEFF6BC2EEFF6CC2EEFF82
:1045D0006DC2EEFFD9D10F0EE615276E286A27BEF1
:1045E0002868070E27C0DBFF080E28C0DBFF070E78
:1045F000DBCFE9FF080EDBCFEAFFD890E936EA36D9
:10460000D890E936EA36720EE926010EEA22EECF9C
:104610006AF2EECF6BF2EECF6CF2EFCF6DF2020EDC
:10462000DB500BE06A0EE66E020EE66E4A0EE66E98
:10463000F8EC0DF0E552E552E552A6D1030E6AC240
:10464000DBFF040E6BC2DBFF050E6CC2DBFF060E48
:104650006DC2DBFF0F0EE615276E286A27BE28689D
:10466000070E27C0DBFF080E28C0DBFF070EDBCFDD
:10467000E9FF080EDBCFEAFFD890E936EA36D8909A
:10468000E936EA36720EE926010EEA22EECF6AF228
:10469000EECF6BF2EECF6CF2EFCF6DF2070EDBCF09
:1046A000E9FF080EDBCFEAFFD890E936EA36D8906A
:1046B000E936EA36720EE926010EEA22030EDBCF56
:1046C000EEFF040EDBCFEEFF050EDBCFEEFF060E96
:1046D000DBCFEEFF020EDB500BE06A0EE66E020E41
:1046E000E66E4A0EE66EF8EC0DF0E552E552E55244
:1046F0004BD10F0EE615276E286A27BE2868070ED5
:1047000027C0DBFF080E28C0DBFF070EDBCFE9FF69
:10471000080EDBCFEAFFD890E936EA36D890E936C2
:10472000EA36720EE926010EEA226EC2EEFF6FC271
:10473000EEFF70C2EEFF71C2EEFF26D10F0EE6153E
:10474000276E286A27BE2868070E27C0DBFF080EE1
:1047500028C0DBFF070EDBCFE9FF080EDBCFEAFF47
:10476000D890E936EA36D890E936EA36720EE9266C
:10477000010EEA22EECF6EF2EECF6FF2EECF70F2C4
:10478000EFCF71F2020EDB500BE06E0EE66E020E02
:10479000E66E4E0EE66EF8EC0DF0E552E552E5528F
:1047A000F3D0030E6EC2DBFF040E6FC2DBFF050EFB
:1047B00070C2DBFF060E71C2DBFF0F0EE615276E1F
:1047C000286A27BE2868070E27C0DBFF080E28C00E
:1047D000DBFF070EDBCFE9FF080EDBCFEAFFD89047
:1047E000E936EA36D890E936EA36720EE926010E45
:1047F000EA22EECF6EF2EECF6FF2EECF70F2EFCF95
:1048000071F2070EDBCFE9FF080EDBCFEAFFD8908D
:10481000E936EA36D890E936EA36720EE926010E14
:10482000EA22030EDBCFEEFF040EDBCFEEFF050E18
:10483000DBCFEEFF060EDBCFEEFF020EDB500BE010
:104840006E0EE66E020EE66E4E0EE66EF8EC0DF0A3
:10485000E552E552E55298D0030E6AC2DBFF040E22
:104860006BC2DBFF050E6CC2DBFF060E6DC2DBFF09
:1048700072C26AF273C26BF274C26CF275C26DF2EC
:10488000030EDBCF72F2040EDBCF73F2050EDBCF2B
:1048900074F2060EDBCF75F2020EDB500BE06A0EEF
:1048A000E66E020EE66E4A0EE66EF8EC0DF0E5528C
:1048B000E552E552720EE66E020EE66E520EE66E9E
:1048C000F8EC0DF0E552E552E5525ED0030E6AC2F7
:1048D000DBFF040E6BC2DBFF050E6CC2DBFF060EB6
:1048E0006DC2DBFF76C26AF277C26BF278C26CF2FD
:1048F00079C26DF2030EDBCF76F2040EDBCF77F2D6
:10490000050EDBCF78F2060EDBCF79F23DD0E6C2A2
:10491000E2F2E36BE2BFE369E2C2E3F2E26BE26B75
:10492000E7C227F0286A296A2A6A27AE03D02868D6
:1049300029682A68030E27C0DBFF040E28C0DBFFAE
:10494000050E29C0DBFF060E2AC0DBFFD950030F7E
:10495000E96EDACFEAFF0F0EEE16EE6AEE6AEE6A45
:10496000030EDBCF1FF0040EDBCF20F01F50E2134D
:104970002050E3130001010E7D6F06D000017D6B16
:1049800003D002D001D000D00201E5511FE0E5C202
:10499000DFFFF00EDF1407E00F0E9715976FF00E94
:1049A000DF149711976F0F0EDF1407E0F00E9715C5
:1049B000976F0F0EDF149711976F020EDB5006E012
:1049C000600E8A6F97C28CF246EC0DF0165002E131
:1049D000CAEC16F0E66A760EE66E010EE66E19DC9B
:1049E000E552E552E552090EE15C02E2E16AE55268
:1049F000E16EE552E7CFD9FF1200D9CFE6FFE1CF54
:104A0000D9FF080EE126040EDB6A050EDB6A060EEE
:104A1000DB6A070EDB6AE4C227F0286A27BE286833
:104A200027C0DEFF28C0DDFFDECF27F0DDCF28F076
:104A3000030ED89028322732E804FBE11F0EDE1661
:104A4000DD6A070E0201E415276E286A296A2A6AC0
:104A500027AE03D0286829682A68040E27C0DBFF28
:104A6000050E28C0DBFF060E29C0DBFF070E2AC09B
:104A7000DBFFD950040FE96EDACFEAFFEF50EE6AA0
:104A8000EFCFF4FFEE6EEF50F4CFEEFFEF6ED950A4
:104A9000040FE96EDACFEAFFEE6A070EEE16EE6A51
:104AA000EE6AE5C227F0286A296A2A6A27AE03D08F
:104AB000286829682A68D950040FE96EDACFEAFF1E
:104AC0002750EE122850EE122950EE122A50EE1204
:104AD000D950040FE96EDACFEAFF040EE76ED890E2
:104AE000EF36010EEB36020EEB36030EEB36E70621
:104AF000F6E1D950040FE96EDACFEAFFF00EEE16B8
:104B0000EE9EEE6AEE6AE6C227F0286A27BE2868A3
:104B1000020E27C0DBFF030E28C0DBFFD950020FB7
:104B2000E96EDACFEAFF040E0F0B06E0EC52D890E4
:104B3000ED32EF32E806FAE1020EDBCF27F0030E8A
:104B4000DBCF28F0296A2A6A28AE02D029682A68B1
:104B5000D950040FE96EDACFEAFF2750EE12285041
:104B6000EE122950EE122A50EE12DECF27F0DDCFE2
:104B700028F0020E246E256A27C01FF028C020F0FE
:104B80003AEC2FF01FC027F020C028F00101275079
:104B9000005D2850015911E2DECF00F1DDCF01F1B7
:104BA000020E246E256A00C11FF001C120F03AEC0C
:104BB0002FF01FC000F120C001F1DECFE9FFDDCFF3
:104BC000EAFF010EE926000EEA22D890E936EA361D
:104BD000000EE926010EEA22040EDBCFEEFF050EE1
:104BE000DBCFEDFFE66AF90EE66E010EE66E09EC2C
:104BF00021F0E552E552E552080EE15C02E2E16A7D
:104C0000E552E16EE552E7CFD9FF1200D9CFE6FFBA
:104C1000E1CFD9FF070EE126D950040FE66E000E52
:104C2000DA20E66E6F0EE66EDBEC0DF0E552E55233
:104C3000E552FF0801E179D0040EDB5075E0040E67
:104C4000DB500101006F016B700EDE6EDD6A010E3C
:104C5000F36E020EF3CFDBFF030EDB6A040EDBCF35
:104C6000E7FFE79EE746E7CFDBFFDB5000085CE2AB
:104C7000DFCF27F0DF2A010EDBCF28F001E3DB2AAC
:104C800027C08AF23FEC0DF002018B51E66ED9503D
:104C9000050FE96EDACFEAFFE552E750EE6EED6AF6
:104CA000D950050FE96EDACFEAFFEE50ED6EEF6AEC
:104CB000050EDBCF27F0060EDBCF28F0000E2716FF
:104CC000FF0E2816DFCF27F0DF2A010EDBCF28F0FA
:104CD00001E3DB2A27C08AF23FEC0DF002018B5181
:104CE000276E286AD950050FE96EDACFEAFF275000
:104CF000EE122850ED12020EDBCFE9FFDB2A030E85
:104D0000DBCFEAFF01E3DB2AD890E936EA36000E72
:104D1000E926010EEA22050EDBCFEEFF060EDBCF01
:104D2000EDFF040EDB06A1D764D0010EF36E020E78
:104D3000F3CFDBFF030EDB6A0101220EFC6F5E0E78
:104D4000FD6FFCC1F6FFFDC1F7FF0900F5CF27F0AD
:104D50000800F5CF28F0010ED89027362836E8064F
:104D6000FBE127C0DEFF28C0DDFFFCC1F6FFFDC16F
:104D7000F7FF0900F5CF00F10A00F5CF01F1DECF12
:104D800027F0DDCF28F0283404E227500008000E79
:104D900028542FE2020EDBCF29F0DB2A030EDBCFF3
:104DA0002AF001E3DB2AD89029362A360101FC518A
:104DB0002924F66EFD512A20F76E0900F5CF27F061
:104DC0000800F5CF28F0020EDBCFE9FF030EDBCFA2
:104DD000EAFFD890E936EA36000EE926010EEA220B
:104DE00027C0EEFF28C0EDFFDF06010E01E2DB0663
:104DF000C6D7070EE15C02E2E16AE552E16EE552D8
:104E0000E7CFD9FF1200D9CFE6FFE1CFD9FF050EDA
:104E1000E126FE0EDB500DE1040EDB6AE00EF36EC0
:104E2000030EF3CFDBFF080EF36E020EF3CFDBFFB2
:104E30000FD0010EF36E040EF3CFDBFFB00EF36E56
:104E4000030EF3CFDBFF0C0EF36E020EF3CFDBFF8E
:104E5000DE6ADD6ADB50000858E2460EE66E020E9E
:104E6000E66E030EDBCFE6FF5DEC0DF0E552E5529A
:104E7000E552FF0805E10201466947694869496949
:104E8000040EDB501BE0DFCFE9FFDF2A010EDBCF92
:104E9000EAFF01E3DB2AD890E936EA36D890E93612
:104EA000EA36420EE926010EEA2246C2EEFF47C26A
:104EB000EEFF48C2EEFF49C2EEFF1AD0DFCFE9FF96
:104EC000DF2A010EDBCFEAFF01E3DB2AD890E936C7
:104ED000EA36D890E936EA36720EE926010EEA2261
:104EE00046C2EEFF47C2EEFF48C2EEFF49C2EEFFE8
:104EF000040E276E030EDBCFE7FF2750E726030ED5
:104F0000E7CFDBFF020EDB06A5D7050EE15C02E270
:104F1000E16AE552E16EE552E7CFD9FF1200D9CF41
:104F2000E6FFE1CFD9FF030EE126020EDB6A800E19
:104F30000201E415800805E1800EF36E020EF3CF46
:104F4000DBFF0F0EE415DF6EDF500B0801E2BDD072
:104F5000010E99C2DBFFDB50040DF3CFE9FFF4CF64
:104F6000EAFF420EE926010EEA2276C2EEFF77C280
:104F7000EEFF78C2EEFF79C2EEFFDFCF99F2020EAC
:104F8000DB50800815E1240E8A6F99C28CF246EC42
:104F90000DF0760EE66E020EE66E010EDB50040D8D
:104FA000F350B00FE66EF8EC0DF0E552E552E55225
:104FB000020EDBCFE7FF02019951E712020EE7CFA5
:104FC000DBFFDF50040DF3CFE9FFF4CFEAFF420E21
:104FD000E926010EEA22EECF46F2EECF47F2EECFFF
:104FE00048F2EFCF49F2E868461908E1E868471946
:104FF00005E1E868481902E1E86849190BE046C292
:1050000076F247C277F248C278F249C279F2020ECC
:10501000DB8849D00101440EFE6F5E0EFF6FDF504A
:10502000E824020DFE51F324F66EFF51F420F76ED2
:105030000900F5CF46F20800F5CF47F20201486BB0
:10504000496BE80E226E030E236E246A256A46C25F
:105050001DF047C21EF048C21FF049C220F0A5EC67
:105060002EF019C046F21AC047F21BC048F21CC00D
:1050700049F2020146514711481149110AE1800ED7
:10508000766F960E776F980E786F796B020EDB8CC9
:105090000AD046C276F247C277F248C278F249C2D5
:1050A00079F2020EDB8ACAEC16F00201440E976F09
:1050B000020EDBCFE6FF740EE66E030EE66E09EC21
:1050C00021F0E552E552E5520AD0E66A740EE66E2A
:1050D000040EE66E09EC21F0E552E552E552030EAE
:1050E000E15C02E2E16AE552E16EE552E7CFD9FF09
:1050F0001200040120511F0B010801E05BD0205178
:10510000600BE842E842E842E842E842010801E078
:1051100051D0245103E0240501E04CD02151230A51
:1051200048E0010A40E0030A30E0010A25E0240AD1
:1051300022E0070A1FE0010A1CE0030A11E0010A4D
:1051400001E038D00201030EF56F0201730EF66F15
:10515000000EF76F0201FD930201080EFA6F2AD0CC
:105160000201030EF56F0201730EF86F000EF96F66
:1051700021D020D01FD01ED00201030EF56F0201F6
:10518000680EF86F000EF96F15D00201030EF56F6F
:105190000201680EF66F000EF76F0201FD93020127
:1051A000070EFA6F07D00201030EF56F22C46FF0ED
:1051B00001D000D012000001686BC20E696F010EB1
:1051C0006A6F6B6B6C6B6D6B080E6E6F616B606BF7
:1051D0001A0E726E1E0E736E0401000E166F050E0F
:1051E000176F400E146F0401196F080E1A6F050E29
:1051F0001B6F880E186F0401480E1E6F050E1F6F7F
:10520000400E1C6F1200D9CFE6FFE1CFD9FF00019D
:10521000606B040118BF30D0FC0EDBCF27F01951B2
:10522000D880275403E2FC0E19C4DBFF0001606B39
:10523000FC0EDB50605D19E26051EA6A080FE96E0E
:10524000050EEA22EF50E66E6051E76EFD0EDBCFF1
:10525000E9FFFE0EDBCFEAFFE750E926000EEA2267
:10526000E552E750EF6E602BE3D70401400E196F53
:105270001817187D880E18130001605100D0E552F0
:10528000E7CFD9FF1200D9CFE6FFE1CFD9FFE65231
:105290000001615101E02FD0DF6ADF2ADF50276E65
:1052A000286AFF0E271801E1285001E10BD0FD0EFE
:1052B000DBCFE9FFDB2AFE0EDBCFEAFF01E3DB2ACF
:1052C000EF50EBE1DF50276E286AD950FD0FE96EF1
:1052D000FF0EDA20EA6E2750EE5E2850ED5AFD0EE2
:1052E000DBCF62F0FE0EDBCF63F0DFCF66F00001B4
:1052F000676B010E616FE552E552E7CFD9FF1200EF
:10530000D9CFE6FFE1CFD9FFE6520001615101E0BC
:1053100030D0DF6ADF2ADF50276E286AFF0E271899
:1053200001E1285001E10CD0FD0EDBCFF6FFDB2AB6
:10533000FE0EDBCFF7FF01E3DB2A0800F550EAE1C0
:10534000DF50276E286AD950FD0FE96EFF0EDA2074
:10535000EA6E2750EE5E2850ED5AFD0EDBCF62F06C
:10536000FE0EDBCF63F0DFCF66F00001010E676F4A
:10537000616FE552E552E7CFD9FF1200D9CFE6FFC2
:10538000E1CFD9FFE65204011CBF6BD0030E000130
:10539000615D01E1616B615101E163D0020E615D0C
:1053A00006E104011D6B0001030E616F54D061051D
:1053B00052E1400E276E286A6651275C000E28587D
:1053C00003E2400EDF6E02D066C0DFFFDFCF1DF4C8
:1053D000DF50665D666F480E646F050E656F67058A
:1053E00015E1DF5012E062C0F6FF63C0F7FF08006E
:1053F000F55064C0E9FF65C0EAFFEF6E642B000E54
:105400006523622B6323DF06ECD713D0DF5011E056
:1054100062C0E9FF63C0EAFFEF5064C0E9FF65C006
:10542000EAFFEF6E642B000E6523622B6323DF0619
:10543000EDD7665110E104011D51276E286A400E18
:10544000271801E1285004E10001020E616F03D02A
:105450000001030E616F400E04011C171C7D880EB5
:105460001C13E552E552E7CFD9FF12000401205189
:10547000600BE842E842E842E842E842000901E005
:1054800055D02151070A51E00B0A4FE0070A40E0CE
:10549000010A2CE00B0A28E0020A26E0030A22E0B7
:1054A000080A12E0010A0EE00F0A0AE0030A01E00E
:1054B0003CD00201010EF56F0201040EFC6F36D0E4
:1054C00036D834D090D832D00201010EF56F0201E7
:1054D000FE0EF66F020EF76F0201FD930201010E40
:1054E000FA6F24D0A8D822D0F4D820D00201010E1F
:1054F000F56F040124510201F66FF76BFF0EF627DA
:10550000020EF7230201FD930201010EFA6F0ED085
:105510000201010EF56F04012451EA6AFF0FE96EE2
:10552000020EEA2222C4EFFF01D000D01200800E4A
:105530000401205D57E12351030A34E0010A10E021
:10554000030A01E04DD00201010EF56F0201EA0EDF
:10555000F66F5B0EF76F120E0201FA6FFB6B40D015
:105560000201010EF56F04012251F66EF76AD89020
:10557000F636F7369F0EF6265C0EF7220900F5CFB9
:10558000F6F20A00F5CFF7F2020E0201F76AF625ED
:10559000F66EF751F7220900F5CFFAF20A00F5CFBF
:1055A000FBF21ED00201010EF56F04012251F66ECE
:1055B000F76AD890F636F736A30EF6265C0EF72279
:1055C0000900F5CFF6F20A00F5CFF7F2F6C2F6FFC2
:1055D000F7C2F7FF0800F5500201FA6FFB6B00D02D
:1055E0000201FD8312000201010EF56F0F0EE66E3F
:1055F000710EE66E0F0EE66EE0EC2DF0E552E55210
:10560000E552010EE66EFF0EE66E020EE66EE0EC6F
:105610002DF0E552E552E55222C4FEF2040122517A
:1056200004E10201050EFC6F05D00201060EFC6FBD
:10563000DBEC28F012000401286B296B04012051D7
:105640001F0B020A14E0030A0EE0010A01E033D046
:105650000201010EF56F040128810201FDA102D0B3
:105660000401288328D00201010EF56F24D0020125
:10567000010EF56F040124510F0B080DF350286A39
:10568000000F276E040E28222451800B01E0010E2A
:10569000040DF35002012724F86F000E2820F96F43
:1056A000F8C2E9FFF9C2EAFFEF50040B03E004017E
:1056B000010E286F00D00201F5050AE10201280E53
:1056C000F66F040EF76F0201FD930201020EFA6FEE
:1056D00012000401220510E120511F0B00090CE10A
:1056E0000201010EF56F030E0401215D03E10201C9
:1056F000FD8102D00201FD91040122513AE12051C5
:105700001F0B020836E124510F0B000932E00201A1
:10571000010EF56F040124510F0B080DF350286A98
:10572000000F276E040E28222451800B01E0010E89
:10573000040DF35002012724F86F000E2820F96FA2
:10574000030E0401215D07E1840EF8C2E9FFF9C2EE
:10575000EAFFEF6E0ED024AF06D0F8C2E9FFF9C21F
:10576000EAFFEF6A06D0880EF8C2E9FFF9C2EAFF45
:10577000EF6E12006C5002E0000E01D0010E000925
:105780000BE0040100513C0BE842E8420D0802E145
:105790000CD801D040D808D06C5002E0000E01D0E7
:1057A000010E040901E047D81200D9CFE6FFE1CF8E
:1057B000D9FFE6520201F46BF56BFA6BFB6B36EC2A
:1057C0002AF0DF6ADF50276E286A010E275C000E80
:1057D00028581BE20201F55101E017D0F76ADF34C7
:1057E000FE0BF736F66EA90EF6265C0EF7220900C0
:1057F000F5CF27F00800F5CF28F004D028C0FAFF35
:105800002750F96EFBDFDF2ADDD7DDD8E552E55200
:10581000E7CFD9FF1200020E0201F45D0AE196D82B
:10582000040100BD03D0C80E006F02D0880E006FC7
:1058300001D00FD91200040E0201FC5D0AE122C45E
:105840006EFF6E50000803E2050EFC6F02D0030EDF
:10585000FC6F0201F4050AE10BD8040104BD03D07A
:10586000C80E046F02D0880E046F01D0F2D8120067
:10587000D9CFE6FFE1CFD9FF020EE1260201080EE3
:10588000FA5D000EFB5905E2FAC2DEFFFBC2DDFF46
:1058900003D0080EDE6EDD6A040104930491010E4C
:1058A000DB500413DFCF05F4000EDB500201FA5F7A
:1058B000010EDB50FB5B280EF86F040EF96F02013E
:1058C000FDA31ED0D9CFE9FFDACFEAFFEE50ED10ED
:1058D00016E0F6C2F6FFF7C2F7FF0800F550F8C26F
:1058E000E9FFF9C2EAFFEF6E0201F82B000EF9237F
:1058F000F62BF723DF06010E01E2DB06E3D71CD00F
:10590000D9CFE9FFDACFEAFFEE50ED1015E0F6C28D
:10591000E9FFF7C2EAFFEF50F8C2E9FFF9C2EAFF78
:10592000EF6E0201F82B000EF923F62BF723DF06AA
:10593000010E01E2DB06E4D7020EE15C02E2E16A5D
:10594000E552E16EE552E7CFD9FF1200D9CFE6FF6D
:10595000E1CFD9FF020EE126030E04010015E76E28
:10596000010EE7CFDBFF01C4DFFFDE500201FA27A3
:10597000DD50FB23280EF66F040EF76FD9CFE9FF39
:10598000DACFEAFFEE50ED1014E0F6C2E9FFF7C2FD
:10599000EAFFEF50F8C2E9FFF9C2EAFFEF6EF82B19
:1059A000000EF923F62BF723DF06010E01E2DB06DA
:1059B000E5D7020EE15C02E2E16AE552E16EE552F2
:1059C000E7CFD9FF12000201F5510CE10401080EE6
:1059D000016F200E026F040E036F840E006F04012E
:1059E000046F35D0040120AF22D00201FA51040126
:1059F000265D0201FB510401275904E226C4FAF294
:105A000027C4FBF235DF0201010EF46F0401080E1A
:105A1000016F200E026F040E036F800E006F0401F1
:105A2000280E066F040E076FC80E046F10D0020117
:105A3000020EF46F0401056BC80E046F0401080E1A
:105A4000016F280E026F040E036FC80E006F6D9871
:105A500012000201F46B0401080E016F200E026FA8
:105A6000040E036F880E006F0401046B12006DA614
:105A70000FD802D06DB613D80201FC0508E16DBA4B
:105A800006D0686A696A69806988020EFC6F120034
:105A90006D6A696A6D860201010EFC6F12006D6A03
:105AA000696A0201FC6B12004FEF2DF00201FC51FC
:105AB00001E13AD06850040B04E06950040B01E0A6
:105AC0003CD86DB231D06850010B04E06950010B35
:105AD00001E054D86850100B04E06950100B01E04D
:105AE00024D86850400B04E06950400B01E03BD8DB
:105AF0006850200B04E06950200B01E036D8685054
:105B0000020B04E06950020B01E036D8030E0201DB
:105B1000FC5D01E209D06850080B06E06950080BF3
:105B200003E0BAEC2BF068961200698468986D82E5
:105B3000A19AA08A0300A09A12006D9269946894B9
:105B400012000201FDA10ED0F8DF6D840001080EE5
:105B50007B6F070E7C6F7B07000E7C5B7B517C119B
:105B6000FAE16D941200689C120070A003D029EC39
:105B70002DF07090689A1200689212006A6A686A42
:105B80009F0E6B6E7B0E696E6E6A0F0EE66E710E67
:105B9000E66E0F0EE66E14D8E552E552E552160E8B
:105BA000706E68A602D06896FCD76D9829EC2DF02F
:105BB0000201FD910201FE6B0201030EFC6F120057
:105BC000D9CFE6FFE1CFD9FFFD0EDBCFE9FFFE0E17
:105BD000DBCFEAFFFC0EDB5004E0EE6AFC0EDB06D6
:105BE000F9D7E552E7CFD9FF1200120100020200F7
:105BF0000008D8040A000000010200010902430065
:105C000002010080FA0904000001020201000524DB
:105C100000100104240202052406000105240100ED
:105C2000010705820308000209040100020A0000BE
:105C3000000705030240000007058302400000043E
:105C400003090434034D006900630072006F0063B0
:105C5000006800690070002000540065006300685F
:105C6000006E006F006C006F006700790020004933
:105C7000006E0063002E00280355004200570020EC
:105C8000004600690072006D0077006100720065D7
:105C900000200043002000760030002E003100FC80
:105CA0005BFC5B3F5C435C775CF250002A0EF66E57
:105CB000080EF76E000EF86E02010900F550EF6F46
:105CC0000900F550F06F03E1EF6701D03DD0090006
:105CD000F550EA6F0900F550EB6F0900F550EC6FD5
:105CE00009000900F550E96E0900F550EA6E090057
:105CF00009000900F550ED6F0900F550EE6F09003D
:105D00000900F6CFF1F2F7CFF2F2F8CFF3F2EAC2E0
:105D1000F6FFEBC2F7FFECC2F8FF0201ED5302E120
:105D2000EE5307E00900F550EE6EED07F8E2EE07DE
:105D3000F9D7F1C2F6FFF2C2F7FFF3C2F8FF020192
:105D4000EF07000EF05BBFD712001D502202F3CF09
:105D500019F0F4CF1AF02302F3501A26000EF420A3
:105D60001B6E1D502402F3501B26000EF4201C6EE7
:105D70001D502502F3501C261E502202F3501A26F5
:105D8000F4501B22000E1C221E502302F3501B262F
:105D9000F4501C221E502402F3501C261F502202D5
:105DA000F3501B26F4501C221F502302F3501C26D4
:105DB00020502202F3501C261200D9CFE6FFDACF82
:105DC000E6FFE1CFD9FFE2CFDAFFC26AC16AC06A5B
:105DD000FC0EDB407F0B3C0BC26EFB0EDB50C16E3A
:105DE000FC0EDB38F00B300BC112FD0EDB50800BCC
:105DF000C06EFD0EDB380F0B070BC012FD0EDB5023
:105E0000040DF350380BC012FC0EDBAE03D09E9C89
:105E10009D8CF28CC280E552E5CFDAFFE7CFD9FF47
:105E200012000800860162026202E603E603AC0685
:105E30000000FFFFFFFFFFFFAC06F70AF70A2A1179
:105E40002A11531C0807D007AC0DA00FD3141B1543
:105E5000581B841C7427A627B0360E389446F84683
:105E60000852CA533A619E61606D047450C3F0D207
:105E70000000FFFF176A25AE43EF2FF0246C251EAC
:105E8000E86A2522171E20AE4BEF2FF01F6C201E54
:105E9000E86A2022171E0FEC30F020BE5BEF2FF0D7
:105EA00017AE000C1F6C201EE86A20221B6C1C1E03
:105EB000E86A1C22000C17BE52EF2FF01888FF0C66
:105EC0001C6A1B6A1A6A196A200EE76ED8901D3682
:105ED0001E361F36203619361A361B361C3622500F
:105EE000195C23501A5824501B5825501C5809E39C
:105EF0002250195E23501A5A24501B5A25501C5AFE
:105F00001D2AE72EE4D71200D9CFE6FFDACFE6FF4D
:105F1000E1CFD9FFE2CFDAFFE652E652C350DF6E9F
:105F2000010EC4CFDBFFDECF27F0DDCF28F027C086
:105F3000F3FF28C0F4FFE552E552E552E5CFDAFF62
:105F4000E7CFD9FF1200D9CFE6FFDACFE6FFE1CFE6
:105F5000D9FFE2CFDAFFE652E652FC0EDBCFDEFFDE
:105F6000DBCFDDFF010EDB50D76EDF50D66EE55282
:105F7000E552E552E5CFDAFFE7CFD9FF1200D9CFDE
:105F8000E6FFDACFE6FFE1CFD9FFE2CFDAFFFD0E81
:105F9000DB507F0BD56ED76AD66AF294FD0EDBAE6E
:105FA00002D0F28A01D0F29AD58EE552E5CFDAFF1F
:105FB000E7CFD9FF1200D9CFE6FFDACFE6FFE1CF76
:105FC000D9FFE2CFDAFFE6528150DF6EFD0EDBBE75
:105FD000F286DBA002D0F18E01D0F19EE552E552AF
:105FE000E5CFDAFFE7CFD9FF120005D810D8FEECD5
:105FF00006F0FCD712000F0EC112140E6F6E0201D4
:10600000FC6B0201FD6B0201FE6B06EF05F037EC45
:106010002DF06FBE02D056EC2DF0BEEF29F01C6AB9
:106020001B6A100EE76ED8901F3620361B361C36C2
:1060300024501B5C25501C5805E324501B5E255042
:106040001C5A1F2AE72EF0D7120013EE00F023EEA1
:1060500000F0F86A189C56EC2EF051EC30F0F5EC9C
:106060002FF0FBD71200FF0EE350396E1B0E00D04D
:1060700001D0200EE76EE72EFED7392EFAD700D0DA
:106080001200FF0EE350E84E1200000000D000D0D6
:1060900000D0E82EFAD71200C2909D9C1200C28256
:1060A00012001200FFFFFFFFFFFFFFFFFFFFFFFFD8
:1060B000FFFFFFFFFFFFFFFFFFFFFFFFFFFFFFFFF0
:1060C000FFFFFFFFFFFFFFFFFFFFFFFFFFFFFFFFE0
:1060D000FFFFFFFFFFFFFFFFFFFFFFFFFFFFFFFFD0
:1060E000FFFFFFFFFFFFFFFFFFFFFFFFFFFFFFFFC0
:0200000400F00A
:020000040030CA
:0E000000240E3A1E008081000FC00FE00F405A
:020000040020DA
:08000000FFFFFFFFFFFFFFFF00
:00000001FF
